:020000040800F2
:1000000088280020FD01000845610008A54500087A
:100010004161000879040008FD7A00080000000032
:10002000000000000000000000000000C173000894
:10003000490D00080000000039680008C573000879
:100040001702000817020008170200089171000843
:10005000170200081702000817020008170200081C
:10006000170200081702000817020008170200080C
:1000700017020008170200081702000817020008FC
:1000800017020008170200081702000817020008EC
:1000900017020008170200081702000817020008DC
:1000A000697400089974000889740008797400085C
:1000B000A9740008B97400081702000817020008A4
:1000C00017020008170200081702000817020008AC
:1000D00017020008ED7A000817020008170200084E
:1000E00017020008170200081702000800F002F8C3
:1000F00000F074F814A696E8000CB244B344DA4554
:1001000001D100F06BF8BAE80F000FA696E83000B6
:10011000A5EB040504EB0607AAEB0704A7F101070A
:100120004FEA15154FEA3414A4F10104AC4201D38F
:1001300000F054F813F0010F18BFFB1A43F001034D
:1001400000F001F8DBE7184788890000A889000063
:100150000A4410F8013B13F0030408BF10F8014BE8
:100160001D1108BF10F8015B641E05D010F8016B6B
:10017000641E01F8016BF9D1002D15D010F8014B68
:1001800003F00C030C2BA1EB04040ABF10F8013B95
:10019000A4EB8314A4EB032405F1010314F8016B11
:1001A0005B1E01F8016BF9D5914238BF10F8013B95
:1001B000D1D370477047000000230024002500269B
:1001C000103A28BF78C1FBD8520728BF30C148BFBA
:1001D0000B6070471FB51FBD10B510BD00F0CFF804
:1001E0001146FFF7F7FF07F0ADFD00F0EDF803B49F
:1001F000FFF7F2FF03BC00F0F5F800000948804764
:1002000009480047FEE7FEE7FEE7FEE7FEE7FEE7F8
:10021000FEE7FEE7FEE7FEE704480549054A064B10
:100220007047000065740008ED0000088822002077
:10023000882800208824002088240020032A40F2F7
:10024000308010F0030C00F0158011F8013BBCF178
:10025000020F624498BF11F801CB00F8013B38BF90
:1002600011F8013BA2F1040298BF00F801CB38BF9E
:1002700000F8013B11F0030300F04F80083AC0F092
:10028000088051F8043B083A51F804CBA0E8081064
:10029000F5E7121D5CBF51F8043B40F8043BAFF397
:1002A0000080D20724BF11F8013B11F801CB48BFF1
:1002B00011F8012B24BF00F8013B00F801CB48BF27
:1002C00000F8012B70474FF0000200B5134694462A
:1002D0009646203922BFA0E80C50A0E80C50B1F19E
:1002E0002001BFF4F7AF090728BFA0E80C5048BFB2
:1002F0000CC05DF804EB890028BF40F8042B08BF50
:10030000704748BF20F8022B11F0804F18BF00F84B
:10031000012B704770477047704710B5203AC0F006
:100320000B80B1E81850A0E81850B1E81850A0E8C8
:100330001850203ABFF4F5AF5FEA027C24BFB1E861
:100340001850A0E8185044BF18C918C0BDE81040A4
:100350005FEA827C24BF51F8043B40F8043B08BFAD
:100360007047D20728BF31F8023B48BF11F8012B74
:1003700028BF20F8023B48BF00F8012B70477546A4
:1003800000F02CF8AE4605006946534620F0070001
:10039000854618B020B5FFF73FFFBDE820404FF07D
:1003A00000064FF000074FF000084FF0000BAC467E
:1003B000ACE8C009ACE8C009ACE8C009ACE8C009C9
:1003C00021F007018D46704710B50446AFF3008059
:1003D0002046BDE81040FFF70ABF00000048704704
:1003E0001802002001491820ABBEFEE726000200DB
:1003F0007047000080B584B0029000200190029800
:1004000000688068C00770B3FFE7029801688868D9
:1004100020F00100886001F0E7FA0190FFE7029800
:1004200000688068C007E8B1FFE701F0DDFA0199D4
:10043000401A032815D3FFE7029800688068C007B8
:1004400070B1FFE70299886A40F010008862029953
:10045000C86A40F00100C86201208DF80F0006E074
:10046000FFE7DCE7FFE700208DF80F00FFE79DF8CE
:100470000F0004B080BD0000FFE7FEE780B586B046
:10048000059004910392029300200190FFE70198E8
:1004900003990968C97A884213DAFFE70198C0EB2B
:1004A000C00141F6A800C2F2000010F83100800837
:1004B000C00708B1FFE7FFE7FFE7019801300190AF
:1004C000E5E741F65000C2F20000006828B9FFE7F6
:1004D00004980078C007F0B1FFE741F65001C2F27E
:1004E0000001002008600499087800F0FE00087000
:1004F00040F27820C2F2000041F2BC31C2F20001A9
:1005000000F040F907F004FF03980068C07A0599ED
:10051000A1F86009FFE706B080BD000080B58AB091
:100520000890079106920593089820B9FFE70120EB
:100530008DF82700B7E0079820B9FFE701208DF874
:100540002700B0E0069820B9FFE701208DF82700CA
:10055000A9E0059820B9FFE701208DF82700A2E067
:1005600000208DF80F00079800F0A2F820B1FFE7F7
:1005700001208DF8270096E006990878497840EA2E
:100580000120ADF81200089805F0C4FFBDF8120074
:100590000004002809D5FFE7BDF812004042ADF87D
:1005A000120001208DF80F00FFE7069800798DF802
:1005B0001100BDF8120000098DF810009DF813001D
:1005C00000F007019DF8100040EA01108DF81000BE
:1005D0009DF81100014601911F280CD0FFE70198FA
:1005E0003F2816D0FFE701985F2820D0FFE7019849
:1005F0007F282AD037E0BDF81200C0F3C00008F011
:100600006FF8029002984FF07C5108F0FDF80290CC
:1006100030E0BDF81200C0F3810008F061F80290EC
:1006200002984FF07A5108F0EFF8029022E0BDF8FE
:100630001200C0F3420008F053F8029002984FF005
:10064000785108F0E1F8029014E0BDF8120000F0D3
:100650000F0008F045F8029002984FF0765108F02C
:10066000D3F8029006E005990020086001208DF87B
:10067000270018E09DF9100008F032F8029907F001
:1006800047FF02909DF80F0030B1FFE7029900206C
:1006900008F086F90290FFE70298059908600020AB
:1006A0008DF82700FFE79DF827000AB080BD000005
:1006B00082B00090009820B9FFE701208DF8070074
:1006C0000CE000980078282804D1FFE700208DF87E
:1006D000070003E001208DF80700FFE79DF8070001
:1006E00002B0704780B586B00490039102920498DE
:1006F00020B9FFE701208DF817003FE0039820B9EB
:10070000FFE701208DF8170038E0029820B9FFE7D5
:1007100001208DF8170031E0049805F0FBFE0498E5
:10072000039905F00FFE0498BE2106F061F8002041
:100730000190FFE7019808280BDCFFE7049805F01B
:10074000B7FE0299019A8854FFE7019801300190A1
:10075000F0E70298082105F02DFD8DF803009DF8C3
:1007600003000299097A884204D0FFE701208DF83E
:10077000170003E000208DF81700FFE79DF8170031
:1007800006B080BD80B586B004900391039820B96F
:10079000FFE701208DF8170044E003990020C8729C
:1007A000FFE70398F02105F0E5FE012801D0FFE7FF
:1007B0000BE003980499C27A01EBC20105F07AFDBF
:1007C0000399C87A0130C872EBE70398C07A0290A7
:1007D000FFE702981F2818DCFFE700200190FFE7E1
:1007E000019807280CDCFFE70498029900EBC1018F
:1007F000019A00208854FFE7019801300190EFE74B
:10080000FFE7029801300290E3E70398C07A0128DD
:1008100004DBFFE700208DF8170003E002208DF8CD
:100820001700FFE79DF8170006B080BD80B584B0C3
:10083000029001918DF80320029820B9FFE7012072
:100840008DF80F005CE0019820B9FFE701208DF8DA
:100850000F0055E00198FFF72BFF20B1FFE70120C3
:100860008DF80F004CE0029805F054FE02980199B3
:1008700005F068FD0298BE2105F0BAFF029805F068
:1008800017FE029805F014FE029805F011FE8DF88F
:100890000200029805F00CFE8DF80100029805F0A8
:1008A00007FE8DF800009DF803008DF80000029807
:1008B00005F030FE0298019905F044FD02984E21A2
:1008C00005F096FF02989DF8021005F091FF02983E
:1008D0009DF8011005F08CFF02989DF8001005F0BE
:1008E00087FF029805F016FE0298019905F02AFD8F
:1008F0000298482105F07CFF00208DF80F00FFE7EB
:100900009DF80F0004B080BD80B582B000900098C3
:1009100020B9FFE701208DF807000EE0009805F0F0
:10092000F9FD0098CC2105F063FF0098442105F003
:100930005FFF00208DF80700FFE79DF8070002B079
:1009400080BD000080B584B00290029820B9FFE716
:1009500001208DF80F001AE001F046F80190FFE742
:10096000029805F06FFD70B9FFE701F03DF80199BD
:10097000401A40F2EF21884204D3FFE703208DF8AC
:100980000F0004E0ECE700208DF80F00FFE79DF872
:100990000F0004B080BD000080B584B002900191CA
:1009A000029820B9FFE701208DF80F0015E00198AB
:1009B00020B9FFE701208DF80F000EE002980199A1
:1009C00008610199D1F82D20029890478DF8030015
:1009D0009DF803008DF80F00FFE79DF80F0004B0AD
:1009E00080BD000080B586B00490049820B9FFE770
:1009F00001208DF8170026E0049802F015FE41F260
:100A00002C62C2F2000241F2BC30C2F2000002903D
:100A1000106040F27821C2F20001019151604FF460
:100A20000041818140F60001C4F20101016105F03D
:100A30005DFC01980299FFF7A5FE002818BF012070
:100A40008DF81700FFE79DF8170006B080BD000085
:100A500080B584B00290029820B9FFE701208DF89C
:100A60000F0031E0029800F033F88DF807009DF890
:100A7000070070B9FFE70299087840F0010008709C
:100A80000299087800F0FB00087000208DF80F0034
:100A90001AE002990020086202980078C00728B185
:100AA000FFE70299087901300871FFE70299087899
:100AB00040F0040008700299087800F0FE00087009
:100AC00002208DF80F00FFE79DF80F0004B080BDF5
:100AD00080B582B00090009820B9FFE701208DF822
:100AE000070009E000990A6952F8080B1831FFF76E
:100AF000F9FD8DF80700FFE79DF8070002B080BD03
:100B000080B584B00290029820B9FFE701208DF8EB
:100B10000F0033E0029800784008C00720B9FFE7D3
:100B200001208DF80F0029E00298FFF791FF8DF862
:100B300007009DF8070028B1FFE79DF807008DF832
:100B40000F001BE0029B1A6952F8080B03F1180111
:100B50002033FFF7E3FC8DF807009DF8070048B14C
:100B6000FFE702994879013048719DF807008DF838
:100B70000F0003E000208DF80F00FFE79DF80F0045
:100B800004B080BD80B586B00490039102920398B2
:100B900020B9FFE701208DF8170047E0049820B93D
:100BA000FFE701208DF8170040E0049803990861E1
:100BB00003990020C8618861029908684A6803990E
:100BC000CA6188610398FFF783FF8DF807009DF8DD
:100BD000070008BBFFE7049800680299039A92F89F
:100BE0002C20FFF723FE8DF807009DF8070048B979
:100BF000FFE70399087840F00200087000208DF8A4
:100C0000170013E00399087800F0FD0008709DF8C4
:100C100007008DF8170009E00399087800F0FD003F
:100C200008709DF807008DF81700FFE79DF8170082
:100C300006B080BD80B584B002900191029820B9C1
:100C4000FFE701208DF80F0015E0019820B9FFE7BC
:100C500001208DF80F000EE00298019942684B6A5E
:100C600002EBC302FFF78EFF8DF803009DF803002F
:100C70008DF80F00FFE79DF80F0004B080BD000065
:100C800080B586B004908DF80F108DF80E20049872
:100C900020B9FFE701208DF8170050E004980068A4
:100CA000FFF732FE8DF80D009DF80D0028B1FFE72B
:100CB0009DF80D008DF8170041E09DF80F00012808
:100CC0000BD1FFE704980068FFF73CFE8DF80D009C
:100CD0009DF80D008DF8170031E09DF80F000228F7
:100CE00028D1FFE7002002909DF80E0001460191F7
:100CF0001F280CD0FFE701983F280BD0FFE7019891
:100D00005F280AD0FFE701987F280AD00DE05E2017
:100D100002900BE0BC20029008E040F277100290B5
:100D200004E040F2EE20029000E0FFE7029800F0BD
:100D300091FCFFE79DF80D008DF81700FFE79DF887
:100D4000170006B080BD00007047000081B0EFF3CF
:100D5000108072B60090FFE7FEE7000080B584B017
:100D600003900291039800F5FA6041F22C61C2F2FF
:100D7000000149684FF48072FFF760FA039890F819
:100D800092090299C0F34002087800F0FE00104476
:100D900008700398022107F0E1F841F2D340C2F253
:100DA0000000007830B9FFE7039890F89209C00777
:100DB000E8B3FFE741F2D341C2F20001002008701E
:100DC000039AB2F8921921F00101A2F89219019048
:100DD000FFE7019841F22C61C2F200010968C97A6B
:100DE000884223DAFFE703980199009100EB410064
:100DF000B0F8940907F08CFC0099C1EBC10241F6F0
:100E0000A801C2F2000101EBC20290600398019AAE
:100E100000EB4200B0F85C0AC2EBC20201EBC20177
:100E20008881FFE7019801300190D2E7FFE70020B9
:100E300004B080BD85B00390029100208DF80700BA
:100E40000090FFE7039890F82400012804D1FFE701
:100E500002208DF81300C3E00399012081F82400DB
:100E6000FFE7FFE702984068062812D8FFE70398DB
:100E70000068406B029A1168526802EB8202053AE0
:100E80001F2393409843914008430399096848639E
:100E900029E0029840680C2812D8FFE70398006800
:100EA000006B029A1168526802EB8202233A1F23F8
:100EB000934098439140084303990968086311E0FF
:100EC00003980068C06A029A1168526802EB8202B5
:100ED000413A1F239340984391400843039909687E
:100EE000C862FFE7FFE7029800680A2812D3FFE70D
:100EF00003980068C06802990A68896802EB420298
:100F00001E3A072393409843914008430399096888
:100F1000C86010E003980068006902990A6889684F
:100F200002EB420207239340984391400843039900
:100F300009680861FFE702980068102805D0FFE7FC
:100F400002980068112840D1FFE70398006842F238
:100F50000041C4F2010188422DD1FFE703980068E7
:100F600080680002002825D4FFE70398016888689C
:100F700040F40000886002980068102819D1FFE74B
:100F800040F20000C2F2000000684DF68361C4F236
:100F90001B31A0FB0110800C00EB80004000009092
:100FA000FFE7009820B1FFE7009801380090F8E7CC
:100FB000FFE7FFE708E00399886A40F020008862B5
:100FC00001208DF80700FFE7FFE7FFE70399002006
:100FD00081F82400FFE79DF807008DF81300FFE774
:100FE0009DF8130005B0704780B588B006900020CA
:100FF0008DF81700049003900290069820B9FFE73F
:1010000001208DF81F00F4E00698806830B1FFE7FA
:101010000698007D08B1FFE7FFE7FFE70698806AC2
:1010200050B9FFE706990020C862069981F82400AC
:10103000069800F0E3F8FFE70698FFF7DBF98DF874
:1010400017000698806AC006002800F1C480FFE7F8
:101050009DF81700002840F0BE80FFE70698806AE0
:1010600040F0020020F4885006998862069948688A
:10107000CA691043097B40EA410103980843039081
:10108000069881680120B1F5807F019008D0FFE7C4
:10109000069880680138B0FA80F040090190FFE7B7
:1010A00001990498CA0740F48071002A18BF0846C5
:1010B00004900698007D01281ED1FFE70698007B6A
:1010C00070B9FFE7069881694EF20000CFF6FF7015
:1010D00000EB41300499084340F4006004900AE0BA
:1010E0000699886A40F0200088620699C86A40F034
:1010F0000100C862FFE7FFE706980068406820F437
:101100006940049908430699096848600698006890
:1011100080684FF2FD71CFF6E171084003990843F2
:10112000069909688860069881680120B1F5807F7A
:10113000009008D0FFE7069880680138B0FA80F088
:1011400040090090FFE7009800F00100002818BF58
:101150004FF48070B0F5807F09D1FFE706980169F0
:101160000020CFF6F07000EB01500290FFE70698E8
:101170000068C06A20F47000029908430699096863
:10118000C86206980068806840F6FE61CFF61F715D
:101190000840039988420CD1FFE706990020C862F5
:1011A0000698806A40F0010020F0020006998862EB
:1011B00010E00698806A40F0100020F002000699C6
:1011C00088620699C86A40F00100C86201208DF863
:1011D0001700FFE708E00699886A40F0100088626F
:1011E00001208DF81700FFE79DF817008DF81F000C
:1011F000FFE79DF81F0008B080BD000082B001909D
:101200000198006842F20041C4F20101884210D105
:10121000FFE7FFE741F21800C4F20200016841F461
:1012200000710160006800F4007000900098FFE712
:10123000FFE702B07047000080B584B002900298CA
:1012400020B9FFE701208DF80F00E0E0029890F848
:10125000200020B9FFE7029800F0DEF8FFE70298CF
:101260000168086840F00100086000F0BDFB0190D3
:10127000FFE7029800684068C007A8B9FFE700F0E0
:10128000B3FB0199401A0B280DD3FFE70299486A76
:1012900040F4003048620299052081F820000120C6
:1012A0008DF80F00B3E0E4E702980168086820F0C9
:1012B0000200086000F098FB0190FFE702980068C8
:1012C00040688007002815D5FFE700F08DFB0199E5
:1012D000401A0B280DD3FFE70299486A40F400300A
:1012E00048620299052081F8200001208DF80F0046
:1012F0008DE0E3E70298007E012807D1FFE702981E
:101300000168086840F08000086006E00298016803
:10131000086820F080000860FFE70298407E0128FE
:1013200007D1FFE702980168086840F040000860B4
:1013300006E002980168086820F040000860FFE7B6
:101340000298807E012807D1FFE7029801680868AB
:1013500040F02000086006E002980168086820F06C
:1013600020000860FFE70298C07E012807D1FFE750
:1013700002980168086820F01000086006E00298F2
:101380000168086840F010000860FFE70298007FDD
:10139000012807D1FFE702980168086840F00800BB
:1013A000086006E002980168086820F008000860FC
:1013B000FFE70298407F012807D1FFE70298016804
:1013C000086840F00400086006E0029801680868B8
:1013D00020F004000860FFE7029B19685A689868CB
:1013E000D3F80CC040EA0C00D3F810C040EA0C005F
:1013F0005B691843013A1043C861029900204862B2
:10140000029A012182F820108DF80F00FFE79DF865
:101410000F0004B080BD000080B58AB009900020A4
:1014200008900790069005900998006846F20041E0
:10143000C4F20001884239D1FFE7FFE741F21C0006
:10144000C4F20200016841F000710160006800F020
:10145000007004900498FFE7FFE741F21800C4F21F
:101460000200016841F004010160006800F004001E
:1014700003900398FFE74FF400600590002006906A
:10148000079040F60000C4F20100019005A9029106
:1014900000F002F9019802994FF48052059202225D
:1014A00006920322089200F0F7F8FFE70AB080BD29
:1014B00083B0019000208DF80300019890F821007E
:1014C00002280DD0FFE7019904208863FFE7019906
:1014D000002081F82000FFE701208DF80B0021E0BB
:1014E00001980168086820F00E0008600198016802
:1014F000086820F0010008600198C16B026C0120AF
:1015000090404860FFE70199012081F82100FFE742
:101510000199002081F82000FFE79DF803008DF875
:101520000B00FFE79DF80B0003B0704780B588B053
:10153000079000208DF81B00079890F821000228E2
:1015400007D0FFE707990420886301208DF81B006E
:1015500076E007980168086820F00E000860079898
:101560000168086820F001000860079800680821F9
:10157000C4F20201884203D1FFE70120059047E051
:10158000079800681C21C4F20201884203D1FFE7DA
:101590001020049039E0079800683021C4F202015D
:1015A000884204D1FFE74FF4807003902AE0079847
:1015B00000684421C4F20201884204D1FFE74FF4DD
:1015C000805002901BE0079800685821C4F2020185
:1015D000884204D1FFE74FF4803001900CE0079877
:1015E00001686C22C4F202024FF08070914208BF81
:1015F0004FF480100190FFE701980290FFE70298F6
:101600000390FFE703980490FFE704980590FFE735
:1016100005980421C4F2020108600799012081F8AD
:101620002100FFE70799002081F82000FFE70798D5
:10163000406B20B1FFE70798416B8847FFE7FFE762
:101640009DF81B0008B080BD81B000900098806BB1
:1016500001B0704780B584B0039000F0C5F90290E6
:10166000039801900198013048B1FFE740F2122041
:10167000C2F200000178019808440190FFE7FFE7FB
:1016800000F0B2F90299401A0199884201D2FFE7AD
:10169000F6E704B080BD000090B00F900E910020DE
:1016A0000D900990FFE70E9800680D99C84000283A
:1016B00000F07F81FFE70D99012088400C900E9883
:1016C00000680C9908400B900B980C99884240F0E8
:1016D0006C81FFE70E9840680590002851D0FFE725
:1016E000059801283AD0FFE7059802283FD0FFE788
:1016F000059803285FD0FFE70598112832D0FFE74F
:101700000598122838D0FFE705980021C1F2110191
:10171000884236D0FFE705980021C1F212018842C5
:101720002FD0FFE705980021C1F22101884228D07F
:10173000FFE705980021C1F22201884221D0FFE78E
:1017400005980021C1F2310188421AD0FFE70598BF
:101750000021C1F23201884213D02FE00E98C068F8
:1017600009902CE00E98C0680430099027E00E988C
:10177000C0680830099022E00E98C0680C300990CB
:101780001DE00E98806818B9FFE70420099011E069
:101790000E988068012806D1FFE7082009900C9870
:1017A0000F99086105E0082009900C980F9948618D
:1017B000FFE7FFE703E00020099000E0FFE70B9858
:1017C000FF2803D8FFE70F98049003E00F98043038
:1017D0000490FFE7049808900B98FF2804D8FFE7CF
:1017E0000D988000039006E00D996FF01F0000EB4C
:1017F00081000390FFE70398079008980068079A14
:101800000F21914088430999914008430899086045
:101810000E98C079C006002840F1C680FFE7FFE7B8
:1018200041F21800C4F20200016841F001010160B8
:10183000006800F0010006900698FFE70D9820F080
:1018400003000821C4F2010140580A900D9800F0ED
:10185000030081000F2000FA01F10A9888430A90E2
:101860000F9840F60001C4F20101884203D1FFE75E
:101870000020029026E00F9840F60041C4F20101DA
:10188000884203D1FFE70120019018E00F9841F250
:101890000001C4F20101884203D1FFE70220009059
:1018A0000AE00F9941F20042C4F201020420914281
:1018B00008BF03200090FFE700980190FFE7019820
:1018C0000290FFE702980D9901F00301890000FAE8
:1018D00001F10A9808430A900A980D9921F0030132
:1018E0000822C4F2010288500E988079C0060028B0
:1018F00009D5FFE70B9A40F20841C4F201010868DC
:101900001043086008E00B9A40F20841C4F201015C
:10191000086890430860FFE70E98807980060028E9
:1019200009D5FFE70B9A40F20C41C4F201010868A7
:101930001043086008E00B9A40F20C41C4F2010128
:10194000086890430860FFE70E98807980070028B8
:1019500009D5FFE70B9A40F20441C4F2010108687F
:101960001043086008E00B9A40F20441C4F2010100
:10197000086890430860FFE70E988079C00748B177
:10198000FFE70B9A40F20041C4F2010108681043DE
:10199000086008E00B9A40F20041C4F201010868B7
:1019A00090430860FFE7FFE7FFE70D9801300D90D7
:1019B00079E610B07047000082B00190ADF80210D7
:1019C0008DF801209DF8010028B1FFE7BDF8020065
:1019D0000199086105E0BDF8020000040199086161
:1019E000FFE702B07047000042F28420C2F200001C
:1019F0000068704780B58EB00C900C9820B9FFE756
:101A000001208DF8370043E10C9890F83D0040B973
:101A1000FFE70C99002081F83C000C9800F03CF99D
:101A2000FFE70C99242081F83D000C9801680868B4
:101A300020F0010008600C980168086840F400403C
:101A400008600C980168086820F40040086000F005
:101A500081FD0A900C98406848F2A061C0F2010133
:101A600088420BD8FFE70A9948F28042C0F21E0272
:101A70000020914238BF012009900AE00A9940F6FF
:101A80000012C0F23D020020914238BF01200990AF
:101A9000FFE70998012804D1FFE701208DF83700FE
:101AA000F6E00A984DF68361C4F21B31A0FB0110E9
:101AB000800C0B900C980068406820F03F000B9958
:101AC00008430C99096848600C980068006A20F087
:101AD0003F0008900C98406848F2A061C0F20101F4
:101AE000884204D8FFE70B98013007900EE00B986E
:101AF0004FF49671484344F6D351C1F26201A0FB02
:101B00000101012000EB91100790FFE70898079969
:101B100008430C99096808620C980068C0694CF683
:101B2000FF71884306900C98406848F2A061C0F2AB
:101B3000010188421FD8FFE70A9801380C994968CB
:101B40004900B0FBF1F001306FF31F30032803D8D8
:101B5000FFE7042005900BE00A9801380C994968CA
:101B60004900B0FBF1F001306FF31F300590FFE743
:101B7000059804904CE00C98806868B9FFE70A98D3
:101B800001380C99496801EB4101B0FBF1F00130DB
:101B90006FF31F3003900DE00A9801380C994968E3
:101BA00019225143B0FBF1F00130042161F31F30E1
:101BB0000390FFE70398000518B9FFE701200290A2
:101BC00023E00C98806868B9FFE70A9801380C99FF
:101BD000496801EB4101B0FBF1F001306FF31F30B8
:101BE00001900DE00A9801380C9949681922514377
:101BF000B0FBF1F00130042161F31F300190FFE7E9
:101C0000019840F400400290FFE702980490FFE73B
:101C10000698049908430C990968C8610C980068F3
:101C2000006820F0C0000C9B1968DA691B6A1A432F
:101C3000104308600C980068806848F2FF318843C0
:101C40000C9A1168D36812691A43104388600C9883
:101C50000068C06820F0FF000C9B19685A699B69F6
:101C60001A431043C8600C980168086840F00100EE
:101C700008600C99002008640C9A202182F83D101D
:101C80000C9908630C9981F83E008DF83700FFE746
:101C90009DF837000EB080BD80B588B00790002059
:101CA00006900590049003900798006845F2004163
:101CB000C4F20001884240D1FFE7FFE741F218007B
:101CC000C4F20200016841F008010160006800F000
:101CD000080002900298FFE74FF440700390122032
:101CE0000490002005900320069040F60040C4F2C6
:101CF000010003A9FFF7D0FCFFE70421C4F20101B2
:101D000008680190019840F0E0600190019840F06F
:101D10000200019001980860FFE7FFE741F21C0014
:101D2000C4F20200016841F400110160006800F48F
:101D3000001000900098FFE7FFE708B080BD0000AA
:101D400040F21220C2F20000027842F28421C2F274
:101D500000010868104408607047000080B542F236
:101D60000001C4F20201086840F01000086003207E
:101D700000F0D6F80F2000F005F800F07BF8002006
:101D800080BD000080B58CB00B90002004900390C3
:101D90008DF80700FFE741F21C00C4F20200016861
:101DA00041F002010160006800F00200009000981C
:101DB000FFE706A802A900F09DFB0998049004988B
:101DC00020B9FFE700F0C6FB059004E000F0C2FB7D
:101DD00040000590FFE705984DF68361C4F21B3182
:101DE000A0FB01014FF0FF3000EB9140039041F266
:101DF000C070C2F2000040F20041C4F20001016074
:101E000040F2E731C16003994160002101618160C6
:101E1000816101F057FB8DF807009DF8070028BB92
:101E2000FFE741F2C070C2F2000001F04FFC8DF8F4
:101E300007009DF80700C0B9FFE71D2000F04CF82F
:101E40000B980F280CD8FFE70B991D20002200F0FB
:101E50004DF80B9840F21421C2F20001086003E033
:101E600001208DF80700FFE7FFE7FFE79DF8070077
:101E70000CB080BD83B0FFE741F21800C4F202004D
:101E8000016841F001010160006800F0010002906A
:101E90000298FFE7FFE741F21C00C4F2020001686C
:101EA00041F080510160006800F08050019001987D
:101EB000FFE7FFE70421C4F20101086800900098E1
:101EC00020F0E0600090009840F0007000900098D2
:101ED0000860FFE703B0704780B582B08DF8070057
:101EE0009DF9070005F00CFE02B080BD80B586B0FC
:101EF0008DF81700049103920020029005F018FE5F
:101F000002909DF91700019002980499039A04F039
:101F10001BF90146019805F013FE06B080BD0000D4
:101F200080B582B00190019805F02CFE02B080BD12
:101F30002021C4F20E2101200860704780B588B0CE
:101F40000790002006900590049003900290079857
:101F50000190012866D0FFE70198022800F0A580D3
:101F6000FFE70198102840F0B080FFE741F204003D
:101F7000C4F202000068039041F20000C4F20200C3
:101F80000068C00100284CD5FFE70398C0F38341E7
:101F900048F6A220C0F60000405C04909DF80E00B8
:101FA000C007F0B1FFE741F20400C4F2020000688C
:101FB000C0F3404148F6B220C0F60000405C0690F5
:101FC0009DF80E00C00758B1FFE7069941F20020C6
:101FD000C0F27A00B0FBF1F0049948430590FFE7A6
:101FE00007E0049840F60011C0F23D014843059017
:101FF000FFE741F20400C4F202000068400200283A
:1020000003D5FFE7059802900AE0059840004AF6DC
:10201000AB21CAF6AA21A0FB011040080290FFE7FD
:10202000FFE753E041F22000C4F202000068039091
:10203000039800F44070B0F5807F0AD1FFE79DF867
:102040000C008007002804D5FFE74FF40040029001
:102050002AE0039800F44070B0F5007F0DD1FFE74F
:1020600041F22400C4F2020000688007002804D571
:10207000FFE749F64040029015E0039800F44070F5
:10208000B0F5407F0DD1FFE741F20000C4F202003D
:1020900000688003002804D5FFE74FF22440029037
:1020A00000E0FFE7FFE7FFE710E000F065FA41F22C
:1020B0000401C4F20201096801F44042022101EB6B
:1020C0005231B0FBF1F0029000E0FFE7029808B057
:1020D00080BD000080B586B004900020039002907F
:1020E00004980078C007002800F0AC80FFE70020CB
:1020F0008DF8070041F21C00C4F202000068C00025
:10210000002813D4FFE7FFE741F21C00C4F20200ED
:10211000016841F080510160006800F0805000903B
:102120000098FFE701208DF80700FFE747F2000065
:10213000C4F200000068C005002822D4FFE747F27F
:102140000001C4F20001086840F480700860FFF7E5
:102150004BFC0390FFE747F20000C4F20000006868
:10216000C00500280CD4FFE7FFF73EFC0399401A96
:10217000652804D3FFE703208DF817008AE0EAE71B
:10218000FFE741F22000C4F20200006800F4407052
:1021900002900298E0B3FFE702980499496801F4BD
:1021A0004071884234D0FFE741F22001C4F20201BD
:1021B000086820F44070029040F24042C4F242228B
:1021C0000120106000201060029808609DF808004F
:1021D000C007E0B1FFE7FFF707FC0390FFE741F21C
:1021E0002000C4F202000068800700280ED4FFE738
:1021F000FFF7FAFB0399401A41F28931884204D370
:10220000FFE703208DF8170044E0E8E7FFE7FFE76A
:1022100041F22001C4F20201086820F44070049ADF
:102220005268104308609DF80700012809D1FFE7B4
:1022300041F21C01C4F20201086820F080500860DD
:10224000FFE7FFE704980078800700280CD5FFE738
:1022500041F20401C4F20201086820F44040049AEB
:10226000926810430860FFE704980078C0060028D1
:102270000CD5FFE741F20401C4F20201086820F422
:102280008000049AD26810430860FFE700208DF8B0
:102290001700FFE79DF8170006B080BD80B584B039
:1022A00002900191029820B9FFE701208DF80F00FC
:1022B0001BE1019842F20001C4F20201096801F039
:1022C0000701884216D9FFE742F20000C4F202007B
:1022D000016821F00701019A11430160006800F0D4
:1022E00007000199884204D0FFE701208DF80F0014
:1022F000FBE0FFE702980078800700282AD5FFE777
:10230000029800784007002809D5FFE741F2040150
:10231000C4F20201086840F4E0600860FFE7029838
:1023200000780007002809D5FFE741F20401C4F254
:102330000201086840F460500860FFE741F20401C0
:10234000C4F20201086820F0F000029A926810437B
:102350000860FFE702980078C007002860D0FFE718
:102360000298406801280ED1FFE741F20000C4F254
:10237000020000688003002804D4FFE701208DF8E4
:102380000F00B2E021E00298406802280ED1FFE77A
:1023900041F20000C4F2020000688001002804D469
:1023A000FFE701208DF80F009FE00DE041F20000F3
:1023B000C4F2020000688007002804D4FFE701206F
:1023C0008DF80F0091E0FFE7FFE741F20401C4F24E
:1023D0000201086820F00300029A52681043086066
:1023E000FFF702FB0090FFE741F20400C4F2020095
:1023F000006800F00C0002994968B0EB810F0ED024
:10240000FFE7FFF7F1FA0099401A41F2893188425B
:1024100004D3FFE703208DF80F0066E0E4E7FFE751
:10242000019842F20001C4F20201096801F00701BB
:10243000884216D2FFE742F20000C4F202000168AF
:1024400021F00701019A11430160006800F00700C4
:102450000199884204D0FFE701208DF80F0044E085
:10246000FFE702980078400700280CD5FFE741F20B
:102470000401C4F20201086820F4E060029AD26804
:1024800010430860FFE702980078000700280DD588
:10249000FFE741F20401C4F20201086820F4605031
:1024A000029A126940EAC2000860FFE700F076F87D
:1024B00041F20401C4F202010968C9B20A0948F6EE
:1024C0008A21C0F60001895CC84040F20001C2F2D6
:1024D0000001086040F21420C2F200000068FFF71B
:1024E00051FC00208DF80F00FFE79DF80F0004B0AD
:1024F00080BD000082B00190009101990F2008601A
:1025000041F20400C4F20200016801F00301019AE3
:102510005160016801F0F001019A9160016801F4D5
:10252000E061019AD160006800F46050C008019930
:10253000086142F20000C4F20200006800F00700E7
:102540000099086002B0704740F20000C2F200003B
:102550000068704780B5FFF7F7FF41F20401C4F24D
:1025600002010968C1F3022248F69A21C0F600016F
:10257000895CC84080BD000080B5FFF7E5FF41F2EF
:102580000401C4F202010968C1F3C22248F69A218B
:10259000C0F60001895CC84080BD000086B0002004
:1025A0000590049003900290019041F20400C4F25F
:1025B000020000680590059800F00C0001460091AB
:1025C00000283FD0FFE70098042804D0FFE70098D8
:1025D000082806D037E041F20020C0F27A000190CE
:1025E00037E00598C0F3834148F6B420C0F60000F8
:1025F000405C02909DF81600C007C0B1FFE741F2B1
:102600000400C4F202000068C0F3404148F6C42050
:10261000C0F60000405C0490029841F20021C0F234
:102620007A0148430499B0FBF1F0039007E0029867
:1026300040F60011C0F23D0148430390FFE70398C4
:10264000019006E0FFE741F20020C0F27A0001901D
:10265000FFE7019806B0704780B586B004900498F3
:1026600020B9FFE701208DF817002EE304980078C9
:10267000C007002800F0AE80FFE741F20400C4F27A
:102680000200006800F00C00042813D0FFE741F2BC
:102690000400C4F20200006800F00C0008281BD1FE
:1026A000FFE741F20400C4F202000068C003002802
:1026B00012D5FFE741F20000C4F202000068800377
:1026C000002808D5FFE70498406820B9FFE70120FB
:1026D0008DF81700F9E27CE0FFE704984068B0F558
:1026E000803F09D1FFE741F20001C4F2020108680E
:1026F00040F48030086032E00498406868B9FFE731
:1027000041F20001C4F20201086820F48030086040
:10271000086820F48020086020E004984068B0F544
:10272000A02F0DD1FFE741F20001C4F202010868B9
:1027300040F480200860086840F4803008600CE0B5
:1027400041F20001C4F20201086820F48030086000
:10275000086820F480200860FFE7FFE7FFE7FFE755
:1027600004984068D0B1FFE7FFF73EF90390FFE718
:1027700041F20000C4F202000068800300280CD47B
:10278000FFE7FFF731F90399401A652804D3FFE703
:1027900003208DF8170098E2EAE719E0FFF724F923
:1027A0000390FFE741F20000C4F2020000688003DA
:1027B00000280CD5FFE7FFF717F90399401A6528A1
:1027C00004D3FFE703208DF817007EE2EAE7FFE776
:1027D000FFE7FFE7049800788007002840F18D802C
:1027E000FFE741F20400C4F20200006810F00C0F91
:1027F00013D0FFE741F20400C4F20200006800F0C9
:102800000C00082829D1FFE741F20400C4F20200BD
:102810000068C003002820D4FFE741F20000C4F2A2
:10282000020000688007002809D5FFE704980069C6
:10283000012804D0FFE701208DF8170045E241F29E
:102840000001C4F20201086820F0F800049A5269FD
:1028500040EAC2000860FFE74EE00498006958B300
:10286000FFE70021C4F2422101200860FFF7BCF815
:102870000390FFE741F20000C4F202000068800705
:1028800000280CD4FFE7FFF7AFF80399401A03289C
:1028900004D3FFE703208DF8170016E2EAE741F2C0
:1028A0000001C4F20201086820F0F800049A52699D
:1028B00040EAC20008601EE00021C4F2422100206C
:1028C0000860FFF791F80390FFE741F20000C4F2BF
:1028D00002000068800700280CD5FFE7FFF784F8A6
:1028E0000399401A032804D3FFE703208DF817004B
:1028F000EBE1EAE7FFE7FFE7FFE70498007800076E
:10290000002848D5FFE70498806918B3FFE740F234
:102910008041C4F2422101200860FFF765F803906E
:10292000FFE741F22400C4F202000068800700289B
:102930000CD4FFE7FFF758F80399401A032804D393
:10294000FFE703208DF81700BFE1EAE7012003F05D
:1029500075FF1FE040F28041C4F242210020086070
:10296000FFF742F80390FFE741F22400C4F20200AF
:102970000068800700280CD5FFE7FFF735F80399BA
:10298000401A032804D3FFE703208DF817009CE1C9
:10299000EAE7FFE7FFE7049800784007002840F1E6
:1029A000D880FFE700208DF8070041F21C00C4F238
:1029B00002000068C000002813D4FFE7FFE741F2DF
:1029C0001C00C4F20200016841F0805101600068FF
:1029D00000F0805000900098FFE701208DF807007C
:1029E000FFE747F20000C4F200000068C0050028BD
:1029F00022D4FFE747F20001C4F20001086840F466
:102A000080700860FEF7F0FF0390FFE747F20000D8
:102A1000C4F200000068C00500280CD4FFE7FEF7F0
:102A2000E3FF0399401A652804D3FFE703208DF8DC
:102A300017004AE1EAE7FFE7FFE70498C0680128CA
:102A400009D1FFE741F22001C4F20201086840F019
:102A50000100086031E00498C06868B9FFE741F2FE
:102A60002001C4F20201086820F001000860086833
:102A700020F0040008601FE00498C06805280DD10C
:102A8000FFE741F22001C4F20201086840F00400AF
:102A90000860086840F0010008600CE041F2200185
:102AA000C4F20201086820F001000860086820F004
:102AB00004000860FFE7FFE7FFE7FFE70498C0684E
:102AC000E0B1FFE7FEF790FF0390FFE741F220003F
:102AD000C4F202000068800700280ED4FFE7FEF76A
:102AE00083FF0399401A41F28931884204D3FFE7FA
:102AF00003208DF81700E8E0E8E71BE0FEF774FF1D
:102B00000390FFE741F22000C4F202000068800752
:102B100000280ED5FFE7FEF767FF0399401A41F240
:102B20008931884204D3FFE703208DF81700CCE0F9
:102B3000E8E7FFE79DF80700012809D1FFE741F228
:102B40001C01C4F20201086820F080500860FFE711
:102B5000FFE70498C069002800F0B380FFE741F266
:102B60000400C4F20200006800F00C00082800F025
:102B70008280FFE70498C06902285CD1FFE76021EA
:102B8000C4F2422100200860FEF72EFF0390FFE709
:102B900041F20000C4F202000068800100280CD558
:102BA000FFE7FEF721FF0399401A032804D3FFE74C
:102BB00003208DF8170088E0EAE70498006AB0F572
:102BC000803F0CD1FFE741F20401C4F20201086822
:102BD00020F40030049A926810430860FFE741F245
:102BE0000401C4F20201086820F47410049B1A6AFC
:102BF0005B6A1A43104308606021C4F2422101203D
:102C00000860FEF7F1FE0390FFE741F20000C4F216
:102C100002000068800100280CD4FFE7FEF7E4FE04
:102C20000399401A032804D3FFE703208DF8170007
:102C30004BE0EAE71EE06021C4F242210020086078
:102C4000FEF7D2FE0390FFE741F20000C4F202005B
:102C50000068800100280CD5FFE7FEF7C5FE039948
:102C6000401A032804D3FFE703208DF817002CE057
:102C7000EAE7FFE724E00498C069012804D1FFE7F0
:102C800001208DF8170020E041F20400C4F2020098
:102C900000680290029800F480300499096A884222
:102CA00008D1FFE7029800F470100499496A88423D
:102CB00004D0FFE701208DF8170006E0FFE7FFE7EB
:102CC000FFE700208DF81700FFE79DF8170006B01A
:102CD00080BD000081B0009001B0704781B00090CD
:102CE00001B0704780B582B001900198006800681B
:102CF000C00718B1FFE7012018B936E00120A0BBDA
:102D0000FFE7019800684068C00718B1FFE701209D
:102D100018B929E0012038BBFFE701980068406836
:102D20004007002803D5FFE7012018B90EE0012075
:102D300060B9FFE70198FFF7D1FF019801686FF0D4
:102D40000400486001990420487406E00198FFF7E8
:102D5000C1FF019901204874FFE7019801684868A4
:102D600020F001004860FFE7FFE702B080BD0000EF
:102D700080B584B0029000200190029820B9FFE74E
:102D800001208DF80F0084E00298407C38B9FFE7FD
:102D9000029900200874029800F080F8FFE7029979
:102DA00002204874029800F00BFA38B1FFE702994C
:102DB0000420487401208DF80F006AE0029804F0A6
:102DC0008FF938B1FFE702990420487401208DF88B
:102DD0000F005EE002980168486820F00700486034
:102DE0000298806848B1FFE746F63041C4F200011E
:102DF000086820F001000860FFE746F62C41C4F2A5
:102E00000001086820F46070029A9268104308601C
:102E100002984068013020B1FFE7029840680190B5
:102E200012E00120FFF78AF80190019838B9FFE716
:102E300002990420487401208DF80F0029E00198C0
:102E400001380190FFE7FFE7BDF8060000F00F0032
:102E5000029909688860BDF8040002990968C86091
:102E6000029804F069F938B1FFE702990420487428
:102E700001208DF80F000CE002990020C873029A1F
:102E800001215173029A9173029A51748DF80F00C7
:102E9000FFE79DF80F0004B080BD000080B584B04E
:102EA00003900398006842F60001C4F200018842D2
:102EB00021D1FFE7FFF73CF8FFE741F21C00C4F225
:102EC0000200016841F000610160006800F00060EC
:102ED00002900298FFE740F23C41C4F242210120F7
:102EE00008600320019000221146FEF7FFFF0198C1
:102EF000FEF7F2FFFFE704B080BD000080B588B0A8
:102F0000069005910492002003900290019006988B
:102F100018B1FFE7059820B9FFE701208DF81F00E1
:102F2000A7E0FFE70698007C012804D1FFE7022014
:102F30008DF81F009DE0069901200874FFE7FFE768
:102F4000069902204874049868B9FFE70598C0788C
:102F50000699C87305984078069948730598807853
:102F60000699887312E00598C07804F0A3F80699D2
:102F7000C8730598407804F09DF806994873059841
:102F8000807804F097F806998873FFE70698417BEC
:102F9000827BC07B04F054F9069908730698007B85
:102FA00005990870069804F015F9039003984BF200
:102FB000C531C9F2A211A0FB0110C00A019001980D
:102FC00019284AD3FFE701984AF6AB21CAF6AA218D
:102FD000A0FB0110000940F2A32141430398A0EB9C
:102FE000C11003900698039904F0C2F960B1FFE79D
:102FF000069904204874FFE7069900200874FFE74B
:1030000001208DF81F0034E0069804F0C9F8029002
:103010000298013000B3FFE70298039988421AD260
:10302000FFE7029845F28011C0F2010108440290C6
:103030000698029904F074F960B1FFE7069904203C
:103040004874FFE7069900200874FFE701208DF817
:103050001F000EE0FFE7FFE7FFE706990120487435
:10306000FFE7069900200874FFE700208DF81F0095
:10307000FFE79DF81F0008B080BD000080B588B054
:10308000069005910492002003900290069818B1D2
:10309000FFE7059820B9FFE701208DF81F008AE0BF
:1030A000FFE70698007C012804D1FFE702208DF895
:1030B0001F0080E0069901200874FFE7FFE70699EA
:1030C00002204874049870B9FFE7059908784A7897
:1030D00089784FF461635843C2EB021200EB82001F
:1030E000084403901BE00598007803F0E3FF4FF4D9
:1030F0006161484300900598407803F0DBFF01468A
:103100000098C1EB011100EB8100019005988078D7
:1031100003F0D0FF0146019808440390FFE70698AA
:10312000039904F025F960B1FFE70699042048747B
:10313000FFE7069900200874FFE701208DF81F00C3
:1031400039E006980168486820F005004860069854
:1031500004F026F802900298013000B3FFE70298CD
:10316000039988421AD2FFE7029845F28011C0F213
:103170000101084402900698029904F0D1F860B168
:10318000FFE7069904204874FFE7069900200874B9
:10319000FFE701208DF81F000DE0FFE7FFE706992C
:1031A00001204874FFE7069900200874FFE700201B
:1031B0008DF81F00FFE79DF81F0008B080BD0000DC
:1031C00080B584B0029000200190029820B9FFE7FA
:1031D00001208DF80F0021E002980168486820F076
:1031E00008004860FEF700FC0190FFE702980068C5
:1031F0004068000700280DD4FFE7FEF7F5FB0199B2
:10320000401AB0F57A7F04D9FFE703208DF80F004C
:1032100004E0EBE700208DF80F00FFE79DF80F00BA
:1032200004B080BD80B584B00290029820B9FFE759
:1032300001208DF80F006EE00298406A60B9FFE748
:1032400002984068B0F5827F01D1FFE703E0029960
:103250000020C861FFE705E002990020086102999B
:103260004861FFE7029900208862029890F85100B7
:1032700040B9FFE70299002081F85000029800F061
:103280004FF8FFE70299022081F851000298016887
:10329000086820F040000860029A019211685068A6
:1032A000D2F808C0D36800F482700CF4044C604477
:1032B00003F400631844136903F0020318445369CC
:1032C00003F001031844936903F400731844D369AD
:1032D00003F038031844136A03F080031843926A1A
:1032E00002F40052104308600298016882690420C9
:1032F00000EA1240486002980168C86920F4006042
:10330000C861029900204865029A012182F8511093
:103310008DF80F00FFE79DF80F0004B080BD00009E
:1033200080B58AB00990002008900790069005901B
:103330000998006843F20001C4F20101884248D1B3
:10334000FFE7FFE741F21800C4F20200016841F410
:1033500080510160006800F4805004900498FFE7F9
:10336000FFE741F21800C4F20200016841F00801D1
:103370000160006800F0080003900398FFE7282030
:103380000590022006900320089040F60040C4F209
:103390000100009005A90191FEF77EF900980199BE
:1033A00010220592002206920792FEF775F9FFE7B8
:1033B0000421C4F2010108680290029840F0E06024
:1033C0000290029840F00100029002980860FFE726
:1033D000FFE70AB080BD000081B0009001B07047E7
:1033E00081B0009001B0704785B003900291FFE773
:1033F000039890F83C00012804D1FFE702208DF8E3
:1034000013005BE00399012081F83C00FFE7FFE730
:103410000399022081F83D000398006840680190FC
:103420000398006880680090019820F07000019077
:10343000029801680198084301900198039909686E
:1034400048600398006842F60041C4F201018842D6
:1034500018D0FFE703980068B0F1804F12D0FFE763
:103460000398006840F20041C4F20001884209D08C
:10347000FFE70398006840F60001C4F200018842AB
:103480000ED1FFE7009820F080000090029841687C
:103490000098084300900098039909688860FFE746
:1034A0000399012081F83D00FFE70399002081F88E
:1034B0003C00FFE700208DF81300FFE79DF81300A4
:1034C00005B0704780B582B00090009820B9FFE742
:1034D00001208DF807003FE0009890F83D0040B9CA
:1034E000FFE70099002081F83C00009800F038F8D0
:1034F000FFE70099022081F83D00009951F8040B84
:1035000003F0F0FF0099012081F84600FFE70099E1
:10351000012081F83E00009981F83F00009981F870
:103520004000009981F84100FFE7FFE70099012082
:1035300081F84200009981F84300009981F8440025
:10354000009981F84500FFE70099012081F83D00CE
:1035500000208DF80700FFE79DF8070002B080BD4E
:1035600080B58AB009900998006842F60041C4F21B
:103570000101884235D1FFE7FFE741F21800C4F2AC
:103580000200016841F400610160006800F400601D
:1035900008900898FFE71820029000220592114633
:1035A000FEF7A4FC0298FEF797FC059A19200390F9
:1035B0001146FEF79BFC0398FEF78EFC059A1A2035
:1035C00004901146FEF792FC0498FEF785FC059ADC
:1035D0001B2006901146FEF789FC0698FEF77CFC3E
:1035E0001FE009980068B0F1804F19D1FFE7FFE7AD
:1035F00041F21C00C4F20200016841F001010160C7
:10360000006800F0010007900798FFE71C20019078
:1036100000221146FEF76AFC0198FEF75DFCFFE709
:10362000FFE70AB080BD000083B00190019890F8D8
:103630003D00012804D0FFE701208DF80B0041E098
:103640000199022081F83D000198006842F600418E
:10365000C4F20101884218D0FFE701980068B0F178
:10366000804F12D0FFE70198006840F20041C4F299
:103670000001884209D0FFE70198006840F6000188
:10368000C4F20001884212D1FFE701980068806807
:1036900000F0070000900098062807D0FFE7019887
:1036A0000168086840F001000860FFE706E0019843
:1036B0000168086840F001000860FFE700208DF80D
:1036C0000B00FFE79DF80B0003B0704783B001903B
:1036D000019890F83D00012804D0FFE701208DF803
:1036E0000B0047E00199022081F83D000198016834
:1036F000C86840F00100C8600198006842F60041C7
:10370000C4F20101884218D0FFE701980068B0F1C7
:10371000804F12D0FFE70198006840F20041C4F2E8
:103720000001884209D0FFE70198006840F60001D7
:10373000C4F20001884212D1FFE701980068806856
:1037400000F0070000900098062807D0FFE70198D6
:103750000168086840F001000860FFE706E0019892
:103760000168086840F001000860FFE700208DF85C
:103770000B00FFE79DF80B0003B0704781B000908D
:1037800000980168C86820F00100C860FFE7009851
:103790000068006A41F21111084210D1FFE7009859
:1037A0000068006A40F24441084207D1FFE70098F0
:1037B0000168086820F001000860FFE7FFE7FFE705
:1037C0000099012081F83D00002001B07047000001
:1037D00080B586B00490039100208DF80B00FFE7C0
:1037E000049890F83C00012804D1FFE702208DF8EE
:1037F0001700ABE00499012081F83C00FFE7FFE7E8
:103800000499022081F83D000498006880680190C6
:10381000019820F077000190019820F47F400190FA
:10382000019804990968886003980068009000284E
:1038300072D0FFE7009810286ED0FFE7009820288C
:103840006AD0FFE70098302866D0FFE7009840284C
:1038500055D0FFE70098502837D0FFE70098602840
:1038600040D0FFE7009870280BD0FFE70098B0F534
:10387000805F05D0FFE70098B0F5005F16D052E0FA
:1038800055E004980068039B5A689968DB6803F068
:10389000ADFE0498006880680190019840F07700C0
:1038A0000190019804990968886040E004980068D4
:1038B000039B5A689968DB6803F098FE04980168D6
:1038C000886840F48040886031E004980068039A7A
:1038D0005168D26803F0BAFE04980068502103F0E2
:1038E0009FFE24E004980068039A5168D26803F0B0
:1038F000D5FE04980068602103F092FE17E004985A
:103900000068039A5168D26803F0A0FE049800682A
:10391000402103F085FE0AE00498006803990968D5
:1039200003F07EFE03E001208DF80B00FFE7049911
:10393000012081F83D00FFE70499002081F83C0058
:10394000FFE79DF80B008DF81700FFE79DF81700C3
:1039500006B080BD81B0009001B0704780B584B0E2
:10396000039003980068C06802900398006800699B
:1039700001909DF804008007002824D5FFE79DF8FA
:103980000800800700281DD5FFE7039801686FF045
:103990000200086103990120087703980068806994
:1039A000800720B1FFE70398FFF7D4FF06E00398F4
:1039B00000F0E2F8039800F0E3F8FFE70399002035
:1039C0000877FFE7FFE79DF804004007002825D5AA
:1039D000FFE79DF80800400700281ED5FFE7039881
:1039E00001686FF0040008610399022008770398CA
:1039F0000068806910F4407F04D0FFE70398FFF768
:103A0000A9FF06E0039800F0B7F8039800F0B8F8B3
:103A1000FFE7039900200877FFE7FFE79DF8040020
:103A20000007002824D5FFE79DF8080000070028BC
:103A30001DD5FFE7039801686FF00800086103993E
:103A40000420087703980068C069800720B1FFE769
:103A50000398FFF77FFF06E0039800F08DF80398C6
:103A600000F08EF8FFE7039900200877FFE7FFE7F3
:103A70009DF80400C006002825D5FFE79DF8080042
:103A8000C00600281ED5FFE7039801686FF01000FC
:103A9000086103990820087703980068C06910F44A
:103AA000407F04D0FFE70398FFF754FF06E0039838
:103AB00000F062F8039800F063F8FFE70399002034
:103AC0000877FFE7FFE79DF80400C00778B1FFE73C
:103AD0009DF80800C00748B1FFE7039801686FF040
:103AE00001000861039800F04FF8FFE7FFE79DF839
:103AF00004000006002810D5FFE79DF80800000626
:103B0000002809D5FFE7039801686FF0800008617D
:103B10000398FFF761FCFFE7FFE79DF8040040060C
:103B2000002810D5FFE79DF808004006002809D5B9
:103B3000FFE7039801686FF040000861039800F008
:103B400035F8FFE7FFE79DF804008006002810D550
:103B5000FFE79DF808008006002809D5FFE70398D5
:103B600001686FF0200008610398FFF739FCFFE758
:103B7000FFE704B080BD000081B0009001B0704745
:103B800081B0009001B0704780B582B0019001987B
:103B9000006840F20041C4F20001884203D1FFE70F
:103BA000FEF7CEF8FFE702B080BD000081B00090C4
:103BB00001B0704782B00190ADF8021002B07047BA
:103BC00080B588B00690FFE7FFE70698006850E8E8
:103BD000030F20F4F0700590FFE70599069802683E
:103BE00042E803100028F0D1FFE7FFE7FFE7FFE717
:103BF0000698006850E8050F20F001000490FFE7E8
:103C000004990698026842E805100028F0D1FFE701
:103C1000FFE70698006B012814D1FFE7FFE7FFE7F5
:103C20000698006850E8030F20F010000390FFE7AB
:103C300003990698026842E803100028F0D1FFE7D4
:103C4000FFE7FFE70698006840690006002832D5C4
:103C5000FFE7FFE7FFE70698006850E8050F20F050
:103C600080000290FFE702990698026842E805107A
:103C70000028F0D1FFE7FFE70698806BD0B1FFE79F
:103C80000698816B002048630698806BFDF710FC56
:103C900078B1FFE70698806BFDF7D6FC202807D1A6
:103CA000FFE706991020486403208DF81F004EE0BE
:103CB000FFE7FFE7FFE70698006840694006002835
:103CC00032D5FFE7FFE7FFE70698006850E8050FE9
:103CD00020F040000190FFE701990698026842E851
:103CE00005100028F0D1FFE7FFE70698C06BD0B1C0
:103CF000FFE70698C16B002048630698C06BFDF78C
:103D0000D7FB78B1FFE70698C06BFDF79DFC202834
:103D100007D1FFE706991020486403208DF81F00A3
:103D200015E0FFE7FFE7FFE706990020C884069942
:103D3000C88506994864069A202182F84210069A9E
:103D400082F84110069908638DF81F00FFE79DF87F
:103D50001F0008B080BD000080B586B00490FFE76A
:103D6000FFE70498006850E8030F20F49070039078
:103D7000FFE703990498026842E803100028F0D195
:103D8000FFE7FFE7FFE7FFE70498006850E8050F4B
:103D900020F001000290FFE702990498026842E8CF
:103DA00005100028F0D1FFE7FFE70498006B012819
:103DB00014D1FFE7FFE7FFE70498006850E8030F1E
:103DC00020F010000190FFE701990498026842E892
:103DD00003100028F0D1FFE7FFE7FFE70498006831
:103DE00040694006002832D5FFE7FFE7FFE7049867
:103DF000006850E8050F20F040000090FFE70099B0
:103E00000498026842E805100028F0D1FFE7FFE7B8
:103E10000498C06BD0B1FFE70498C16B00204863E1
:103E20000498C06BFDF744FB78B1FFE70498C06BC2
:103E3000FDF70AFC202807D1FFE704991020486409
:103E400003208DF817000EE0FFE7FFE7FFE7049976
:103E50000020C885049A202182F842100499086342
:103E60008DF81700FFE79DF8170006B080BD000031
:103E700080B584B00290FFE7FFE70298006850E841
:103E8000030F20F0C0000190FFE70199029802683B
:103E900042E803100028F0D1FFE7FFE7029800682E
:103EA00040690006002832D5FFE7FFE7FFE70298E8
:103EB000006850E8050F20F080000090FFE70099AF
:103EC0000298026842E805100028F0D1FFE7FFE7FA
:103ED0000298806BD0B1FFE70298816B00204863A5
:103EE0000298806BFDF7E4FA78B1FFE70298806BE7
:103EF000FDF7AAFB202807D1FFE7029910204864AC
:103F000003208DF80F000CE0FFE7FFE7FFE70299C1
:103F10000020C884029A202182F841108DF80F00F9
:103F2000FFE79DF80F0004B080BD000081B0009055
:103F300001B0704780B592B0119011980068006888
:103F4000109011980068C0680F901198006840693F
:103F50000E9000200D900C90109800F00F000D9026
:103F60000D9888B9FFE79DF84000800600280AD523
:103F7000FFE79DF83C008006002804D5FFE7119874
:103F800003F024FCE9E1FFE70D98002800F0C2806F
:103F9000FFE79DF83800C00738B9FFE7BDF83C00DF
:103FA00010F4907F00F0B680FFE79DF84000C00756
:103FB00058B1FFE79DF83D00C00730B1FFE7119908
:103FC000486C40F001004864FFE79DF8400040075E
:103FD00000280BD5FFE79DF83800C00730B1FFE798
:103FE0001199486C40F002004864FFE79DF84000DA
:103FF000800700280BD5FFE79DF83800C00730B1D7
:10400000FFE71199486C40F004004864FFE79DF811
:1040100040000007002811D5FFE79DF83C0080060E
:10402000002805D4FFE79DF83800C00730B1FFE74E
:104030001199486C40F008004864FFE71198406C03
:10404000002866D0FFE79DF84000800600280AD5CA
:10405000FFE79DF83C008006002804D5FFE7119893
:1040600003F0B4FBFFE7119800684069C0F38010CB
:104070000C901198406C0007002804D4FFE70C98BE
:1040800000283ED0FFE7119803F042FB119800682A
:104090004069400600282FD5FFE7FFE7FFE71198AA
:1040A000006850E8050F20F040000B90FFE70B99E7
:1040B0001198026842E805100028F0D1FFE7FFE7F9
:1040C0001198C06B98B1FFE71198C16B47F2F1608E
:1040D000C0F6000048631198C06BFDF727FA28B1BD
:1040E000FFE71198C06B416B8847FFE703E0119829
:1040F000FFF71CFFFFE703E01198FFF717FFFFE74B
:1041000006E01198FFF712FF119900204864FFE7BD
:10411000FFE722E11198006B012840F0FE80FFE7E5
:104120009DF84000C006002840F1F780FFE79DF8A9
:104130003C00C006002840F1F080FFE7FFE70020C8
:104140000A901198006800680A9011980068406809
:104150000A900A98FFE71198006840694006002815
:1041600040F18180FFE71198C06B00684068ADF8AE
:104170002600BDF82600002874D0FFE7BDF8260011
:104180001199898D88426DDAFFE7BDF826001199F3
:10419000C8851198C06B8069202858D0FFE7FFE7D9
:1041A000FFE71198006850E8030F20F48070089032
:1041B000FFE708991198026842E803100028F0D13F
:1041C000FFE7FFE7FFE7FFE71198006850E8050FFA
:1041D00020F001000790FFE707991198026842E874
:1041E00005100028F0D1FFE7FFE7FFE7FFE7119890
:1041F000006850E8050F20F040000690FFE70699A0
:104200001198026842E805100028F0D1FFE7FFE7A7
:104210001199202081F84200119900200863FFE7DE
:10422000FFE71198006850E8030F20F01000059098
:10423000FFE705991198026842E803100028F0D1C1
:10424000FFE7FFE71198C06BFDF732F9FFE711991F
:10425000022048631198818DC28D891A89B2FFF7B7
:10426000A9FCFFE779E01199888DC98D401AADF856
:1042700012001198C08D00284ED0FFE7BDF8120043
:10428000002849D0FFE7FFE7FFE71198006850E8F2
:10429000030F20F490700390FFE7039911980268D0
:1042A00042E803100028F0D1FFE7FFE7FFE7FFE750
:1042B0001198006850E8050F20F001000290FFE718
:1042C00002991198026842E805100028F0D1FFE732
:1042D000FFE71199202081F842001199002008631E
:1042E000FFE7FFE71198006850E8030F20F0100087
:1042F0000190FFE701991198026842E80310002835
:10430000F0D1FFE7FFE71199022048631198BDF84B
:104310001210FFF74FFCFFE71FE09DF8400000067A
:1043200000280AD5FFE79DF83C000006002804D5C8
:10433000FFE7119803F090FB0FE09DF84000400666
:1043400000280AD5FFE79DF83C004006002804D568
:10435000FFE7119803F026FAFFE712B080BD0000D6
:1043600080B582B00090009820B9FFE701208DF859
:10437000070040E00098806908B1FFE700E0FFE730
:10438000009890F8410040B9FFE70099002081F8BB
:104390004000009800F034F8FFE70099242081F8ED
:1043A000410000980168C86820F40050C860009877
:1043B00003F0C2FA00980168086920F4904008618F
:1043C00000980168486920F02A0048610098016857
:1043D000C86840F40050C860009900204864009A02
:1043E000202182F84110009A82F842100099486317
:1043F0008DF80700FFE79DF8070002B080BD0000C0
:1044000080B58CB00B9000200A900990089007901E
:104410000B98006843F60001C4F20101884251D1B3
:10442000FFE7FFE741F21800C4F20200016841F41F
:1044300080410160006800F4804006900698FFE724
:10444000FFE741F21800C4F20200016841F00801E0
:104450000160006800F0080005900598FFE7402023
:1044600007900220089003200A9040F60040C4F212
:104470000100029007A90391FDF70EF90298039934
:1044800080220792002208920992FDF705F9FFE7C2
:104490000421C4F2010108680490049840F0E0602F
:1044A0000490049840F00400049004980860FFE72A
:1044B0002520019000221146FDF718FD0198FDF717
:1044C0000BFDFFE70CB080BD80B584B00290019178
:1044D000ADF80220029890F84200202817D1FFE79B
:1044E000019820B1FFE7BDF8020020B9FFE70120E5
:1044F0008DF80F000FE002990020086302980199DF
:10450000BDF8022003F076FA8DF80F0003E00220D8
:104510008DF80F00FFE79DF80F0004B080BD00008C
:1045200081B0009001B0704784B002900191ADF865
:104530000220029890F84100202826D1FFE7019838
:1045400020B1FFE7BDF8020020B9FFE701208DF898
:104550000F001EE0019802990862BDF8020002995E
:104560008884BDF802000299C8840299002048643A
:10457000029A212182F8411002990A68D16841F01B
:104580008001D1608DF80F0003E002208DF80F004C
:10459000FFE79DF80F0004B07047000081B0009065
:1045A00001B07047FFE7FEE783B0ADF80800ADF853
:1045B0000610ADF80420ADF80230BDF80800BDF8D3
:1045C0000410884215DBFFE7BDF80800BDF80410B1
:1045D000401ABDF806100844BDF80210884204DDF8
:1045E000FFE702208DF80B0007E000208DF80B009C
:1045F00003E002208DF80B00FFE79DF80B0003B0ED
:104600007047000080B586B084460898CDF810C089
:10461000ADF80E10ADF80C2002938DF80700BDF830
:104620000C00B0F5FA6F04DDFFE703208DF81700EA
:1046300027E0BDF80E00BDF80C1000224FF47A738D
:10464000FFF7B2FF78B9FFE7BDF80E00C0F30B111A
:1046500040F27830C2F2000000EB410000F6621038
:104660000499086003E002208DF8170009E0BDF806
:104670000E0000F00F000299088000208DF817004E
:10468000FFE79DF8170006B080BD000080B584B03C
:104690000290ADF80610ADF804208DF80330BDF897
:1046A00004007E2804DBFFE703208DF80F0049E0BB
:1046B0009DF80300E8B9FFE7BDF80600BDF8041057
:1046C00000224FF4FA63FFF76FFF68B9FFE7BDF808
:1046D000061040F27830C2F2000000EB410000F614
:1046E00094100299086003E002208DF80F0029E081
:1046F00024E09DF8030001281BD1FFE7BDF8060068
:10470000BDF8041000224FF4FA63FFF74DFF58B9CB
:10471000FFE7BDF8061040F27830C2F2000000EB6F
:1047200041000299086003E002208DF80F0009E0C3
:1047300003E001208DF80F0004E0FFE700208DF872
:104740000F00FFE79DF80F0004B080BD84B0039018
:10475000029100208DF80700009002984078082808
:1047600003D1FFE70120009018E0029840782B2841
:1047700003D1FFE7002000900FE00298407800F09E
:104780007F000E2803D8FFE70120009004E0029884
:10479000007B02300090FFE7FFE7FFE7009807305B
:1047A0000090009804B0704740F69C61C2F200018E
:1047B0000720086048F6C620C0F6000048600122C5
:1047C0008A6048F6CC20C0F60000C8600A614861E3
:1047D0008A61C8610A6248628A62C86270470000E2
:1047E00041F29C21C2F2000100200880887088807C
:1047F000C880088148818881C881088248827047C2
:1048000041F29C21C2F20001888801308880704703
:1048100041F29C20C2F20000408A4FF6FE718842AD
:104820000CDCFFE741F29C21C2F20001488A013012
:104830004882088840F001000880FFE770470000C8
:1048400041F29C20C2F20000C0884FF6FE718842FF
:1048500008DCFFE741F29C21C2F20001C888013068
:10486000C880FFE77047000041F29C20C2F20000C0
:1048700000894FF6FE71884208DCFFE741F29C2177
:10488000C2F20001088901300881FFE7704700008B
:1048900041F29C20C2F2000040894FF6FE7188422E
:1048A00008DCFFE741F29C21C2F200014889013097
:1048B0004881FFE77047000041F29C20C2F20000EF
:1048C000C0894FF6FE71884208DCFFE741F29C2167
:1048D000C2F20001C8890130C881FFE770470000BB
:1048E00041F29C20C2F2000080894FF6FE7188429E
:1048F00008DCFFE741F29C21C2F200018889013007
:104900008881FFE77047000041F29C20C2F200005E
:104910008078704780B586B004900498C089ADF85F
:104920000E000498008AADF80C0041F29C20C2F2FF
:1049300000008078012809D1FFE7BDF80E000128AA
:1049400004D0FFE700208DF8170025E1BDF80E0028
:1049500001460291142800F20E810299DFE811F05D
:10496000150021004C005B0068000B010B010B01DE
:104970000B010B0172007F008E009D00AC00BB009C
:10498000CA00D900E8000B01F700BDF80E00049939
:10499000C881BDF80C0004990882049904200873AA
:1049A000F6E041F29C21C2F2000100208870BDF8BF
:1049B0000C00B0F57F4F03D1FFE7FFF711FF0FE0C9
:1049C00041F29C21C2F200010091002001908880F8
:1049D000C880088148818881C88108824882FFE7B1
:1049E000BDF80E000499C881BDF80C000499088236
:1049F000049904200873CBE0BDF80E000499C88127
:104A000041F29C20C2F200000088049908820499B7
:104A100004200873BCE00499487840F08000487096
:104A20000499012081F8080100208DF81700B3E0F7
:104A300041F29C21C2F200010120887000208DF813
:104A40001700A9E0FFF7CCFEBDF80E000499C8815D
:104A500004990020088204990420087398E0BDF8A6
:104A60000E000499C88141F29C20C2F200008088A7
:104A70000499088204990420087389E0BDF80E00A7
:104A80000499C88141F29C20C2F20000C0880499B8
:104A900008820499042008737AE0BDF80E00049996
:104AA000C88141F29C20C2F200000089049908826A
:104AB0000499042008736BE0BDF80E000499C881C6
:104AC00041F29C20C2F200004089049908820499B6
:104AD000042008735CE0BDF80E000499C88141F21F
:104AE0009C20C2F200008089049908820499042065
:104AF00008734DE0BDF80E000499C88141F29C2076
:104B0000C2F20000C0890499088204990420087345
:104B10003EE0BDF80E000499C88141F29C20C2F22B
:104B20000000008A049908820499042008732FE089
:104B3000BDF80E000499C88141F29C20C2F2000029
:104B4000408A0499088204990420087320E041F205
:104B50009C22C2F2000200205082118821F0010143
:104B60001180BDF80E10049AD1810499088204992D
:104B7000042008730CE00499487840F080004870E5
:104B80000499012081F8080100208DF8170003E046
:104B900001208DF81700FFE79DF8170006B080BDD3
:104BA00080B58AB008900020ADF81A00089A1189E3
:104BB00052896B46186007A80DF11A03FFF722FD12
:104BC000089981F80801089890F8080120B1FFE7DA
:104BD00000208DF827008AE008994889013800EB09
:104BE0005072012000EBD20008730020ADF81800CD
:104BF000ADF81600ADF81400ADF81200BDF81A10AB
:104C000003910290FFE70298BDF81A10089A5289A2
:104C10001144013901EB1172012101EB221188428B
:104C20004EDCFFE70020ADF81800FFE703980F28DF
:104C30001ADCFFE70399012000FA01F1BDF8180022
:104C40000843ADF81800BDF812000130ADF81200AD
:104C500080B208994989884201DBFFE704E0FFE759
:104C6000039801300390E1E7002003900798029A2F
:104C700030F81200BDF818100840BDF81A10C840EE
:104C8000089901EB4201C8810298012813DBFFE774
:104C90000798029930F81100BDF818201040000460
:104CA000BDF81A2040FA02F2089800EB4101888909
:104CB00010438881FFE7FFE7029801300290A2E7E6
:104CC000FFE7029800280ED4FFE70898029900EB4E
:104CD0004101CA89100A40EA0220C881FFE7029810
:104CE00001380290EDE701208DF82700FFE79DF8DD
:104CF00027000AB080BD000080B584B00290029900
:104D0000822008710298C078013801460191032879
:104D100031D80199DFE801F0021222270298807948
:104D200020B9FFE7029900208871FFE7029802216D
:104D300000F072FE02990320C87120E00298807989
:104D400020B9FFE7029903208871FFE70298062146
:104D500000F062FE02990420C87110E0029903205D
:104D600081F808010BE00298817900F055FE029964
:104D70000120C87103E000208DF80F000CE00298BC
:104D800090F8080120B1FFE700208DF80F0003E044
:104D900001208DF80F00FFE79DF80F0004B080BDE3
:104DA00080B584B0029002980189428901A800234D
:104DB000FFF76CFC029981F80801029890F808014D
:104DC00020B1FFE700208DF80F001EE0029948890E
:104DD0004000087300200090FFE70098029949897D
:104DE00088420EDAFFE70198811C01910088029940
:104DF000009A01EB4201C881FFE700980130009062
:104E0000EBE701208DF80F00FFE79DF80F0004B0DD
:104E100080BD000080B584B002900298018942896B
:104E200001A80123FFF732FC029981F808010298DA
:104E300090F8080120B1FFE700208DF80F002FE067
:104E4000029948894000087300200090FFE700980D
:104E50000299498988421FDAFFE70198B0F90000FA
:104E600001280ADBFFE70198811C01910088029963
:104E7000009A01EB4201C88109E00198811C01916F
:104E800000880299009A01EB4201C881FFE7FFE721
:104E9000009801300090DAE701208DF80F00FFE75D
:104EA0009DF80F0004B080BD80B58AB008900899C5
:104EB000087B4989013901EB5172012101EBE201C3
:104EC000884208D0FFE70899032081F808010020F4
:104ED0008DF82700A2E00020ADF81A00089801899B
:104EE00042896B460120186007A80DF11A03FFF7ED
:104EF00089FB089981F80801089890F8080120B109
:104F0000FFE700208DF8270088E00020ADF81800AA
:104F10000590ADF81200ADF81000BDF81A1003911D
:104F20000290FFE70298BDF81A10089A52891144BE
:104F3000013901EB1172012101EB2211884269DC78
:104F4000FFE70020ADF81800FFE703980F281ADCF0
:104F5000FFE70399012000FA01F1BDF818000843AA
:104F6000ADF81800BDF810000130ADF8100080B2A7
:104F700008994989884201DBFFE704E0FFE70398CD
:104F800001300390E1E7002003900798029930F880
:104F90001100ADF812000898029900EB4100C08999
:104FA00040BABDF81A1088400590029801280FDB1E
:104FB000FFE70898029900EB4100808940BABDF8EC
:104FC0001A1000FA01F1059840EA21400590FFE728
:104FD0000598BDF8181008400799029A21F81200A8
:104FE000BDF81200BDF8181020EA01030799029AD3
:104FF00031F81200184321F81200BDF8100008998A
:105000004989884201DBFFE704E0FFE702980130AD
:10501000029087E701208DF82700FFE79DF8270021
:105020000AB080BD80B584B0029002984189007BAF
:10503000B0EB410F08D0FFE70299032081F8080187
:1050400000208DF80F002DE002980189428901A807
:105050000023FFF71BFB029981F80801029890F8E2
:10506000080120B1FFE700208DF80F001AE00020B2
:105070000090FFE700980299498988420EDAFFE71D
:105080000298009900EB4100C08901998A1C0192A5
:105090000880FFE7009801300090EBE701208DF8D1
:1050A0000F00FFE79DF80F0004B080BD80B586B00B
:1050B00004900498408970B1FFE704984089B0F5E6
:1050C0007F4F08D0FFE70499032081F808010020F2
:1050D0008DF8170036E00022ADF80A200498018907
:1050E0006B460120186003A80DF10A03FFF78AFA46
:1050F000049981F80801049890F8080120B1FFE7AD
:1051000000208DF817001DE004984089B0F57F4F0E
:105110000AD1FFE7BDF80A10012000FA01F2039955
:1051200008881043088009E0BDF80A10012000FA41
:1051300001F20399088890430880FFE701208DF869
:105140001700FFE79DF8170006B080BD80B584B05A
:1051500002900298018901A801220023FFF796FA24
:10516000029981F80801029890F8080120B1FFE740
:1051700000208DF80F0007E002984089019908800F
:1051800001208DF80F00FFE79DF80F0004B080BDEF
:1051900080B58AB008900791069200200590089883
:1051A00090F82100C00760B1FFE7089890F8201040
:1051B0000020B0EBD11F04D0FFE70898C06805902D
:1051C000D4E0079800780699059A531C05938854F3
:1051D000079840780699059A531C059388540798B8
:1051E00090F90100002800F1B780FFE707984078A8
:1051F0002B284FD1FFE7079880780699059A531C12
:10520000059388540798C0780699059A531C05930E
:105210008854079800790699059A531C0593885479
:10522000079840790699059A531C05938854079866
:1052300080790699059A531C059388540798C0797C
:105240000699059A531C059388540798007BFB2800
:1052500004DBFFE707208DF82700B0E007980E3049
:10526000049000200390FFE703980799097B884288
:105270000FDAFFE7049800780699059A531C059306
:105280008854049801300490FFE70398013003909C
:10529000EAE760E00798407808281DD1FFE7079803
:1052A000C07B0699059A531C059388540798C089BA
:1052B0000699059A531C059388540798407C0699D3
:1052C000059A531C059388540798008A0699059AF5
:1052D000531C059388543DE00798007BFA2808DCAE
:1052E000FFE70798007B0699059A531C059388549D
:1052F00003E007208DF8270061E007980E30029048
:1053000000200190FFE701980799097B884220DA85
:10531000FFE7019800EBD07121F00101401A40B97C
:10532000FFE7029840780699059A531C0593885424
:105330000AE0029800780699059A531C0593885450
:10534000029802300290FFE7FFE7019801300190D8
:10535000D9E7FFE7FFE708E0079890F8080106990A
:10536000059A531C05938854FFE7FFE70598B0F1B1
:10537000FF3F04DCFFE707208DF827001FE00698B9
:10538000059902F01DFCADF80200BDF80200079976
:10539000A1F80A019DF802000699059A531C05938D
:1053A00088549DF803000699059A531C0593885468
:1053B00005980899C86001208DF82700FFE79DF83F
:1053C00027000AB080BD000080B58AB00890079120
:1053D000069200200490089A92F8201001F0BF0174
:1053E00082F82010039006980499405C0899097887
:1053F000884207D0FFE70799002008700498013021
:10540000049007E0069804994A1C0492405C0799AE
:105410000870FFE7069804994A1C0492405C0799BB
:105420004870079840780006002809D5FFE7FFF785
:1054300043FA07990020087005208DF827001EE127
:10544000079840782B2819D1FFE7069804994A1C41
:105450000492405C07998870069804994A1C04924B
:10546000405C0799C870069804994A1C0492405CF5
:105470000799887107990020087350E007984078D1
:10548000082828D1FFE7069804994A1C0492405C3A
:1054900000020799C881069804994A1C0492425C4C
:1054A0000799C8891043C881069804994A1C049238
:1054B000405C000207990882069804994A1C0492ED
:1054C000425C0799088A10430882079900200881E6
:1054D0000799488122E0069804994A1C0492405C8E
:1054E000000207990881069804994A1C0492425CBC
:1054F0000799088910430881069804994A1C049268
:10550000405C000207994881069804994A1C04925D
:10551000425C0799488910434881FFE7FFE70898F4
:10552000406840780F2806D0FFE708984068407828
:10553000102809D1FFE7069804994A1C0492405CA0
:1055400008994968087304E00898416800200873C6
:10555000FFE708980799FFF7F9F803900898C068E3
:10556000039988420BDAFFE7089991F8200040F090
:10557000400081F8200005208DF827007FE0089882
:10558000C0680399884206DDFFE7FFF759F9082054
:105590008DF8270073E0FFE70798007B002840D0D4
:1055A000FFE70798007BFB280BDBFFE707994878AC
:1055B00040F080004870FFF743F908208DF827007D
:1055C0005DE007980E30029000200190FFE70198FF
:1055D0000799097B884223DAFFE7019800EBD07135
:1055E00021F00101401A48B9FFE7069804994A1CC6
:1055F0000492405C0002029908800CE0069804992D
:105600004A1C0492425C0299088810430880029860
:1056100002300290FFE7FFE7019801300190D6E7E2
:10562000FFE70698049902F0CBFAADF8020006985D
:1056300004994A1C0492405C0799A1F80A01069853
:1056400004994A1C0492425C0799B1F80A0140EAA5
:105650000220A1F80A010798B0F80A01BDF802106B
:10566000884208D0FFE7FFF7EBF80799487840F049
:1056700080004870FFE701208DF82700FFE79DF8C4
:1056800027000AB080BD000080B586B00490039169
:1056900000208DF80B00049991F8200000F07F00A5
:1056A00081F82000049991F8210000F0FE0081F8B3
:1056B0002100049991F8200000F0F70081F8200003
:1056C000049991F8200000F0DF0081F82000FFF736
:1056D00097F80498007820B1FFE70398007868B93C
:1056E000FFE7FFF7FDF80499052081F828000498EA
:1056F000039901F079F98DF8170088E1FFF7C8F8F0
:10570000039890F90100002800F15181FFE7039808
:1057100040780138014601912A2800F21F81019941
:10572000DFE811F02B001C013A004900580082000C
:105730001C010D011C011C011C011C011C011C0190
:10574000AC00D5001C011C011C011C011C011C012A
:105750001C011C011C011C011C011C011C011C0161
:105760001C011C011C011C011C011C011C011C0151
:105770001C011C011C011C01FE0004984068FFF77D
:105780000FFA0246049991F8200000F07F0040EAE9
:10579000C21081F82000E6E004984068FFF700FBA3
:1057A0000246049991F8200000F07F0040EAC21000
:1057B00081F82000D7E004984068FFF72BFB0246F1
:1057C000049991F8200000F07F0040EAC21081F8AF
:1057D0002000C8E004984068FFF768FC024604997E
:1057E00091F8200000F07F0040EAC21081F820000C
:1057F000049890F820100020B0EBD11F13D0FFE7E1
:10580000049991F8210040F0040081F821000499E6
:1058100091F8210040F0010081F821000499C86846
:105820000238C860FFE79EE004984068FFF78EFCEE
:105830000246049991F8200000F07F0040EAC2106F
:1058400081F82000049890F820100020B0EBD11FC0
:1058500013D0FFE7049991F8210040F0040081F88B
:105860002100049991F8210040F0010081F8210005
:105870000499C8680238C860FFE774E0049840687B
:10588000FFF712FB0246049991F8200000F07F0018
:1058900040EAC21081F82000049890F820100020FF
:1058A000B0EBD11F12D0FFE7049991F8210040F02E
:1058B000040081F82100049991F8210040F00100D2
:1058C00081F8210004990620C860FFE74BE00498A6
:1058D0004068FFF7A7FB0246049991F8200000F00A
:1058E0007F0040EAC21081F82000049890F8201050
:1058F0000020B0EBD11F12D0FFE7049991F82100EE
:1059000040F0040081F82100049991F8210040F052
:10591000010081F8210004990620C860FFE722E019
:1059200004984068FFF7E8F90246049991F82000CE
:1059300000F07F0040EAC21081F8200013E00498D4
:105940004068FEF7E7FF0246049991F8200000F056
:105950007F0040EAC21081F8200004E00399012092
:1059600081F80801FFE7FEF7CFFF01280DD1FFE71F
:10597000FEF7B6FF0499052081F8280004980399E2
:1059800001F032F88DF8170041E0049890F82010EB
:105990000020B0EBD11F08D1FFE7FEF765FF0399A8
:1059A000487840F08000487000E0FFE7FFE7049887
:1059B00090F82000C008C00728B1FFE70498012133
:1059C00000F05AFFFFE7049890F821004008C00754
:1059D00038B9FFE70498039901F03CF88DF80B0003
:1059E0000BE00498039900F0FFFF049991F821005F
:1059F00000F0FD0081F82100FFE79DF80B000499FD
:105A000081F828009DF80B008DF81700FFE79DF83E
:105A1000170006B080BD000080B58AB009900891DB
:105A200040F69C60C2F200000790099880790690C9
:105A30000999002081F8080105900490FFE7049877
:105A4000F9281EDCFFE70698FF2801D3FFE718E0DE
:105A50000498023004900798069950F83110049881
:105A6000084404900498F92804DCFFE70698013004
:105A70000690FFE706980899884201D9FFE700E001
:105A8000DDE706980138059009980E300390002054
:105A90000290099880790190FFE701980599884262
:105AA00013D8FFE701980399029A531C0293885474
:105AB00003980799019A01EBC20202A900F028F8A5
:105AC000FFE7019801300190E7E701980138019064
:105AD0000998007BA8B1FFE7029809990873059817
:105AE00001300999887101980899884204D1FFE72B
:105AF00009990020487103E00999FF204871FFE7E8
:105B000004E00999032081F80801FFE70AB080BD8D
:105B100084B0039002910192019800680399DDF826
:105B200008C0DCF80020531CCCF80030885400205A
:105B30000090FFE7009801990968884212D2FFE7B8
:105B4000019840680099405C0399DDF808C0DCF8D2
:105B50000020531CCCF800308854FFE70098013037
:105B60000090E7E704B0704784B002908DF807100A
:105B7000ADF804208DF80330029820B9FFE701202A
:105B80008DF80F002EE09DF8030098B9FFE79DF80F
:105B90000700012805DBFFE79DF80700F82804DB74
:105BA000FFE701208DF80F001CE09DF80700029927
:105BB000087003E0029900200870FFE7BDF80400B8
:105BC000029948839DF8030020B1FFE70299032062
:105BD000087603E0029901200876FFE700208DF89F
:105BE0000F00FFE79DF80F0004B0704780B584B048
:105BF000029001910092029818B1FFE7019820B934
:105C0000FFE701208DF80F0022E0FEF7CDFD02999D
:105C100003200870029941F28830488302990120DC
:105C2000087602980199009A002300F03BFF029940
:105C300081F82800029890F82800012804D1FFE795
:105C400000208DF80F0003E001208DF80F00FFE722
:105C50009DF80F0004B080BD80B584B00290019122
:105C6000029820B9FFE701208DF80F002EE002987E
:105C7000007E032804DBFFE701208DF80F0025E0FC
:105C8000FEF7AEFD019840B1FFE70298019900F0E0
:105C900053FF029981F828000AE0029841F2B021EE
:105CA000C2F2000100F048FF029981F82800FFE7E6
:105CB000029890F82800012804D1FFE700208DF811
:105CC0000F0003E001208DF80F00FFE79DF80F00A3
:105CD00004B080BD80B584B000220392029201928C
:105CE00041F2D450C2F20000009042F20041C4F2EE
:105CF0000101016082600121017302754FF460238C
:105D0000C36142600161FBF76FF918B1FFE7FBF770
:105D10001DF8FFE711200190012002900020039060
:105D200041F2D450C2F2000001A9FBF783F818B188
:105D3000FFE7FBF70BF8FFE704B080BD80B582B04A
:105D400041F20460C2F20000009046F20041C4F249
:105D50000001016010214160002101918160C1605A
:105D600001614161017641768176C17601774177A3
:105D7000FBF762FA18B1FFE7FAF7E8FFFFE702B0B6
:105D800080BD000080B592B00020119010900F905F
:105D90000E90FFE741F21800C4F20200016841F0E2
:105DA00010010160006800F010000D900D98FFE7F1
:105DB000FFE741F21800C4F20200016841F020013F
:105DC0000160006800F020000C900C98FFE7FFE7EE
:105DD00041F21800C4F20200016841F004010160C0
:105DE000006800F004000B900B98FFE7FFE741F21A
:105DF0001800C4F20200016841F008010160006867
:105E000000F008000A900A98FFE741F20000C4F28F
:105E1000010001904FF40051009100220592FBF720
:105E2000CBFD059A40F60000C4F20100029048F252
:105E3000FE710391FBF7C0FD059A40F60040C4F2E5
:105E4000010007904FF607410991FBF7B5FD009A55
:105E5000019805990E92012204920F92109102214D
:105E6000069111910EA90891FBF716FC0298049B6C
:105E7000059A08990E930F921092FBF70DFC029869
:105E8000DDF810C0059B069A0899DDF80CE0CDF806
:105E900038E0CDF83CC010931192FBF7FDFBDDF824
:105EA00010C0059B069A07980899DDF824E0CDF804
:105EB00038E0CDF83CC010931192FBF7EDFB12B027
:105EC00080BD000080B582B041F24060C2F20000A7
:105ED000019045F20041C4F20001016048F2A06166
:105EE000C0F20101416000218160C1604FF4804235
:105EF000026141618161C1610162FBF77BFD18B103
:105F0000FFE7FAF723FFFFE702B080BD80B582B05C
:105F100000208DF80600ADF80400009041F2C46046
:105F2000C2F2000042F60001C4F2000101604FF02D
:105F3000FF3141604FF440718160FCF719FF18B1E7
:105F4000FFE7FAF703FFFFE700208DF804008DF864
:105F500005008DF8060041F2C460C2F2000001A9FC
:105F60000122FDF78BF818B1FFE7FAF7EFFEFFE724
:105F700001228DF800208DF801208DF802200020EC
:105F80008DF8030041F2C460C2F200006946FCF7DC
:105F9000B5FF18B1FFE7FAF7D9FEFFE702B080BD01
:105FA00080B582B041F2D860C2F20000019043F2A5
:105FB0000001C4F2010101604FF4827141600021CF
:105FC0008160C160016141614FF400728261082209
:105FD000C2610162416281620A21C162FDF722F958
:105FE00018B1FFE7FAF7B2FEFFE702B080BD00008C
:105FF00080B588B000210091079106910591049128
:106000000391029141F23070C2F20000019042F619
:106010000042C4F201020260416081604FF6FF72EB
:10602000C260016141618161FDF74CFA18B1FFE77F
:10603000FAF78CFEFFE74FF48050049041F2307085
:10604000C2F2000004A9FDF7C3FB18B1FFE7FAF79D
:106050007DFEFFE700200290039041F23070C2F213
:10606000000002A9FDF7C0F918B1FFE7FAF76EFECC
:10607000FFE708B080BD000080B588B00021019125
:1060800007910691059104910391029141F2787074
:10609000C2F200004FF08042026041F61F424260AF
:1060A00081604FF6FF72C26001618161FDF70AFAFB
:1060B00018B1FFE7FAF74AFEFFE74FF4805004906B
:1060C00041F27870C2F2000004A9FDF781FB18B11B
:1060D000FFE7FAF73BFEFFE700200290039041F252
:1060E0007870C2F2000002A9FDF77EF918B1FFE74F
:1060F000FAF72CFEFFE708B080BD000080B582B043
:1061000041F60800C2F2000001900121016343F64C
:106110000001C4F2010101604FF4E131416000214E
:106120008160C16001610C2242618161C161FEF741
:1061300017F918B1FFE7FAF709FEFFE702B080BDD3
:10614000FFE7FEE7FFE7FEE788B0079006910592BC
:10615000079800F0070004900498C0F10700052894
:1061600003D3FFE70420019004E00498C0F1070086
:106170000190FFE70198039004980430062803D8A3
:10618000FFE70020009003E0049803380090FFE749
:106190000098029006980399012202FA01F1013950
:1061A0000840029B984005999A40013A11400843E3
:1061B00008B0704783B002908DF8071000208DF86A
:1061C0000600FFE79DF80700411E8DF80710A0B3F9
:1061D000FFE70298411C029100788DF80500082025
:1061E0008DF80400FFE79DF8040028B3FFE79DF851
:1061F00006009DF80510484000F001008DF80300EE
:106200009DF8060040088DF806009DF803209DF8D3
:10621000060080F08C01002A18BF08468DF80600A1
:106220009DF8050040088DF80500FFE79DF8040083
:1062300001388DF80400D6E7C4E79DF8060003B0E6
:106240007047000086B00590059840F20C21C2F21C
:10625000000109684843049042F62440C4F201005A
:106260000068ADF80E0000200290BDF80E00ADF8F9
:106270000600FFE702980499884218D2FFE742F629
:106280002440C4F201000068ADF80400BDF8040029
:10629000BDF80610401AADF80200BDF802100298D1
:1062A00008440290BDF80400ADF80600E2E706B02D
:1062B0007047000083B00290019100208DF8030028
:1062C000FFE79DF8030007280EDCFFE702989DF822
:1062D00003201044C07801998854FFE79DF803001B
:1062E00001308DF80300ECE703B0704780B584B04F
:1062F000039003980121019100F05CF80199039843
:1063000000F042F84FF47A700090FFF79BFF03987B
:106310000021029100F038F80098FFF793FF0199EF
:10632000039800F031F84FF4FA60FFF78BFF029802
:106330000399087003998870039948700399C8728B
:1063400004B080BD80B584B00390029103985521BC
:1063500000F04EFA00208DF80700FFE79DF80700D7
:1063600007280EDCFFE7039802999DF80720895C57
:1063700000F03EFAFFE79DF8070001308DF80700B6
:10638000ECE704B080BD000082B001908DF80310EE
:106390009DF8030028B1FFE7019988890969086120
:1063A00005E001998889000409690861FFE702B0E6
:1063B0007047000083B002908DF8071002980069C2
:1063C0000430009040F20820C2F2000001680F2063
:1063D00000FA01F200990868904308609DF80700F0
:1063E00098B9FFE740F20820C2F2000001680820D7
:1063F00000FA01F2009908681043086002980169E8
:10640000C86840F40040C8600CE040F20820C2F2C6
:1064100000000168022000FA01F2009908681043A8
:106420000860FFE703B0704781B0009000980069F2
:106430008068009989890840002818BF012001B0B0
:106440007047000080B586B00390039820B9FFE73D
:1064500000208DF8130026E0EFF3108072B605904F
:10646000002101918DF80B100398FFF78DFF039821
:106470000121FFF79FFF0220FFF7E4FE0199039837
:10648000FFF798FF0620FFF7DDFE0398FFF7CCFF2C
:106490008DF80B003220FFF7D5FE62B69DF80B0099
:1064A0008DF81300FFE79DF8130006B080BD0000D3
:1064B00080B584B00290029820B9FFE700208DF8E3
:1064C0000F0022E000208DF8070008208DF806005C
:1064D000FFE79DF80600411E8DF8061080B1FFE72A
:1064E0009DF8070040088DF807000298FFF7AAFF03
:1064F00001469DF8070040EAC1108DF80700E8E763
:106500009DF807008DF80F00FFE79DF80F0004B01D
:1065100080BD000080B584B00290029820B9FFE7EA
:1065200001208DF80F0021E0029800210091FFF773
:106530002BFF02980121FFF73DFF4FF4F070FFF7AA
:1065400081FE00990298FFF735FF4620FFF77AFE9B
:106550000298FFF769FF8DF807004FF4CD70FFF741
:1065600071FE9DF807008DF80F00FFE79DF80F0002
:1065700004B080BD80B586B004908DF80F100498EB
:1065800020B9FFE700208DF81700E6E001208DF824
:106590000E0000218DF80D108DF80C108DF80B10E9
:1065A0008DF80A0004988078002840F0BF80FFE74B
:1065B0000498FFF7AFFF50B1FFE70499002008707F
:1065C00004998870049948708DF81700C5E0049804
:1065D0009DF80F1000F00CF9FFE70498FFF732FF69
:1065E0008DF809000498FFF72DFF8DF808009DF83D
:1065F0000900012806D1FFE79DF80800012801D114
:10660000FFE77DE09DF809009DF80810884205D05D
:10661000FFE79DF809008DF8070034E09DF80E00B3
:106620000499097888420FDAFFE704989DF80C1066
:106630000844C0789DF80A10014000200029C8BF16
:1066400001208DF807000AE09DF80E0004990978F2
:10665000401AB0FA80F040098DF80700FFE79DF876
:10666000070078B9FFE79DF80E008DF80D009DF842
:106670000D00082805DCFFE79DF80D00049948701F
:10668000FFE7FFE7FFE79DF8070001280AD1FFE7D2
:106690009DF80A2004989DF80C100144C878104316
:1066A000C87009E09DF80A2004989DF80C10014478
:1066B000C8789043C870FFE704989DF8071000F071
:1066C00051F89DF80E0001308DF80E009DF80A007B
:1066D00040008DF80A009DF80A0048B9FFE79DF8D0
:1066E0000C0001308DF80C0001208DF80A00FFE746
:1066F000FFE7FFE79DF80C000828FFF66EAFFFE705
:106700009DF80E00412810DBFFE79DF80D0004996D
:1067100008700498007820B9FFE704990120887078
:10672000FFE701208DF80B00FFE7FFE79DF80B0066
:1067300020B1FFE70498C07850B9FFE70499002022
:10674000087004998870049948708DF80B00FFE771
:106750009DF80B008DF81700FFE79DF8170006B0B5
:1067600080BD000080B586B004908DF80F100498AD
:1067700008B9FFE73AE0EFF3108072B605909DF894
:106780000F00C0B1FFE7049800210291FFF7FCFD64
:1067900004980121FFF70EFE0820FFF753FD029930
:1067A0000498FFF707FE3220FFF74CFD029904988A
:1067B000FFF700FE18E0049800210191FFF7E4FDC7
:1067C000049801210091FFF7F5FD3920FFF73AFD0C
:1067D00001990498FFF7EEFD0098FFF733FD01994A
:1067E0000498FFF7E7FDFFE762B6FFE706B080BD5C
:1067F00080B582B001908DF80310019808B9FFE7C9
:1068000017E008208DF80200FFE79DF80200411E06
:106810008DF8021068B1FFE701989DF8031001F0B0
:106820000101FFF79FFF9DF8030040088DF803006A
:10683000EBE702B080BD00007047000082B001901D
:10684000019840F20001C2F200010968C90844F64B
:10685000D352C1F26202A1FB022189094843009090
:10686000FFE700BFFFE70098411E00910028F8D124
:10687000FFE702B07047000080B584B003908DF848
:106880000B1000208DF80A00039800F039FA9DF8EB
:106890000B004007002844D4FFE79DF80B00800759
:1068A000002823D5FFE703980069FDF755FA8DF816
:1068B0000A00039991F8200000F0FD0081F8200003
:1068C000039991F8200000F0BF0081F8200003999F
:1068D00091F8200000F0FB0081F82000039991F866
:1068E000200000F0EF0081F82000FFE79DF80B008A
:1068F000C007A8B1FFE703980069FDF7B9FA8DF862
:106900000A00039991F8200000F0F70081F82000B8
:10691000039991F8200000F0DF0081F82000FFE7E4
:1069200042E003980069FDF74BF98DF80A0000205A
:106930000190FFE70198B0F5817F0ADCFFE703983B
:106940008168019A00208854FFE701980130019086
:10695000F0E7039991F8200000F0FD0081F8200095
:10696000039991F8200000F0BF0081F820000399FE
:1069700091F8200000F0FB0081F82000039991F8C5
:10698000200000F0EF0081F82000039991F820002A
:1069900000F0F70081F82000039991F8200000F042
:1069A000DF0081F82000FFE70399032081F8280029
:1069B00004B080BD80B584B002900191009202982D
:1069C000007E022808DCFFE702980199009AFEF792
:1069D000DFFB8DF80F0003E002208DF80F00FFE7CA
:1069E0009DF80F0004B080BD80B584B00390029183
:1069F00000208DF807000398007E014600910128D1
:106A00000CD0FFE7009802280FD0FFE7009803287A
:106A100016D1FFE7039800F04DF9FFE703980299BC
:106A200000F08AF88DF807000AE0039991F8200039
:106A300000F0FE0081F8200001208DF80700FFE73C
:106A40009DF80700012801D0FFE7FFE79DF8070048
:106A500004B080BD80B584B00390029100208DF811
:106A600007000398007E0138022807D8FFE7039843
:106A7000029900F075F98DF80700FFE79DF807000F
:106A800001280BD0FFE70398007E022805DCFFE712
:106A900003980299FFF7A8FFFFE7FFE79DF80700BB
:106AA00004B080BD85B003900291019200930398D9
:106AB00020B9FFE702208DF813001FE0029820B9EB
:106AC000FFE702208DF8130018E00298039908618F
:106AD0000198039948610398806838B9FFE70399E2
:106AE00041F2D030C2F20000886003E000980399C0
:106AF0008860FFE701208DF81300FFE79DF8130081
:106B000005B0704780B584B0029001910092029860
:106B1000007E022808DCFFE702980199009AFEF740
:106B200053FC8DF80F0003E002208DF80F00FFE703
:106B30009DF80F0004B080BD80B584B00290019133
:106B400000208DF803008DF80200029890F82000D4
:106B50008008C00720B1FFE704208DF80F004DE04A
:106B6000029991F8200040F0010081F8200002997C
:106B700091F8200040F0040081F82000029991F87B
:106B8000200000F0EF0081F8200001980299486091
:106B9000029890F820008009C00720B9FFE7029909
:106BA0000020C860FFE7029800690168C86840F0EB
:106BB0001000C86002988168C2680069114440F200
:106BC0000312FDF781FC8DF802009DF8020038B138
:106BD000FFE702980421FFF74FFE8DF8030003E062
:106BE00001208DF80300FFE79DF80300029981F86A
:106BF00028009DF803008DF80F00FFE79DF80F00B7
:106C000004B080BD80B584B0029001910298007EEE
:106C1000032804DBFFE702208DF80F0006E002984E
:106C20000199FEF731FD8DF80F00FFE79DF80F0089
:106C300004B080BD80B582B001900198406908B968
:106C4000FFE734E001984069FCF788FE01980421D1
:106C5000FFF712FE0199062081F828000198007EB6
:106C6000022809DCFFE70199486800780978884222
:106C700001D1FFE7FFE7FFE70198007E032811DB62
:106C8000FFE7019991F8200000F0FE0081F8200054
:106C90000198C06928B1FFE701984168C26990472F
:106CA000FFE704E001984168FFF79EFEFFE702B0AE
:106CB00080BD000080B582B0019001984069D8B1D4
:106CC000FFE7019840690168002048620198408B05
:106CD00088B1FFE70199488B49690968C862019842
:106CE0004069FCF7F3FC019991F8200040F00200A4
:106CF00081F82000FFE7FFE7012002B080BD00001F
:106D000080B582B0019001984069A8B1FFE7019871
:106D1000408B28B1FFE701984069FCF72FFDFFE7A2
:106D20000198406901680020486201984069016843
:106D30006FF001000861FFE7012002B080BD000094
:106D400081B000900098406930B1FFE70098406939
:106D5000016800204862FFE7012001B07047000091
:106D600080B584B00290019100208DF803008DF869
:106D70000200029890F82000C008C00720B1FFE789
:106D800004208DF80F005DE0029801998268FFF7FA
:106D900011FE8DF803009DF80300012809D0FFE7DC
:106DA00002980421FFF768FD02984168FFF71CFE76
:106DB0003EE0029991F8200040F0010081F82000A7
:106DC000029991F8200040F0080081F82000029913
:106DD00091F8200000F0DF0081F82000019802996E
:106DE00048600298C06800280ADCFFE70298042186
:106DF000FFF742FD8DF8030002208DF80F0021E01F
:106E0000029A916810699289FDF78EFB8DF8020055
:106E10009DF8020038B1FFE702980421FFF72CFD2E
:106E20008DF8030003E001208DF80300FFE7FFE782
:106E30009DF80300029981F828009DF803008DF861
:106E40000F00FFE79DF80F0004B080BD80B582B051
:106E500001900198006908B9FFE700E1019991F8F4
:106E6000210040F0080081F82100019800690068C5
:106E70000068C006002840F1A580FFE7019800697E
:106E80000068C068C006002840F19C80FFE7FFE76B
:106E90000020009001980069006800680090019847
:106EA00000690068406800900098FFE70198006959
:106EB000FDF740F8019991F8200000F0BF0081F83B
:106EC0002000019890F820008008C007002878D0A2
:106ED000FFE7019890F820004008C007002870D014
:106EE000FFE701980169888DC98D421A0199C86828
:106EF0001044C8600198C068012861DBFFE7019871
:106F00000069FCF729FF019991F8200000F0FD00CD
:106F100081F82000019991F8200000F0BF0081F86D
:106F20002000019991F8200000F0FB0081F820007A
:106F3000019991F8200000F0EF0081F820000199FC
:106F400091F8200040F0100081F82000019841687D
:106F50008268FFF7D7FD019981F82800019890F821
:106F60002800012826D1FFE70198FFF7C9FE42F269
:106F70008420C2F200000068019948620198007EF6
:106F8000022805DCFFE701984168FFF73BFE10E0AF
:106F9000019991F8200000F0FE0081F8200001988E
:106FA000C06928B1FFE701984168C2699047FFE7CF
:106FB000FFE704E001984168FFF716FDFFE7FFE7F0
:106FC000FFE74CE001980069FCF7B4FFFFE7019888
:106FD0000069406C80BBFFE701980069C08D0130FB
:106FE00001990969898D88420BD1FFE7019890F8D2
:106FF00020008008C00720B1FFE70198FFF75AFE84
:10700000FFE70198FFF79CFE01980069C08C90B9DA
:10701000FFE7019890F82000C008C00758B1FFE7CB
:107020000198006990F84100212804D0FFE70198F9
:1070300000F018F8FFE712E001980069406C0007C3
:10704000002803D5FFE7FDF7E3FBFFE701980421E4
:10705000FFF712FC01984168FFF7C6FCFFE702B09A
:1070600080BD000080B582B0019001208DF8030042
:1070700000208DF80200019991F8200000F0F7003F
:1070800081F82000019991F8200000F0DF0081F8DC
:107090002000019991F8200040F0200081F82000A4
:1070A00001984168FFF7A0FC8DF803009DF80300EC
:1070B00002B080BD82B08DF80700002000909DF8DE
:1070C0000700000900EB80004000009000989DF848
:1070D000071001F00F010844C0B202B07047000071
:1070E00080B584B0029000200190FAF77DFC0190F9
:1070F000FFE7029800684068800600280DD4FFE78B
:10710000FAF772FC0199401AB0F57A7F04D9FFE7CB
:1071100003208DF80F000AE0EBE702980168486849
:1071200040F01000486000208DF80F00FFE79DF848
:107130000F0004B080BD000080B584B00290002034
:10714000019002980168486820F010004860FAF742
:107150004BFC0190FFE70298006840688006002819
:107160000DD4FFE7FAF740FC0199401AB0F57A7F99
:1071700004D9FFE703208DF80F0004E0EBE70020BF
:107180008DF80F00FFE79DF80F0004B080BD0000F0
:1071900080B541F2C460C2F20000FBF7A3FD80BDE0
:1071A00082B001900020ADF80200ADF80000019817
:1071B0000068006AADF8020001980068406AADF806
:1071C0000000BDF80210BDF8000040EA014002B026
:1071D0007047000084B003900020ADF80A00ADF8BD
:1071E0000800ADF806000090039800688069ADF8CB
:1071F0000A0003980068C069ADF8060003980068AB
:107200008069ADF80800BDF80A00BDF80810884292
:107210000AD0FFE7BDF8081003980068C06980B283
:1072200040EA0140009007E0BDF80A10BDF80600F2
:1072300040EA01400090FFE7009804B0704700006A
:1072400084B003908DF80B108DF80A200020019077
:107250000090039800F5FA6001909DF80B00022859
:107260002DD8FFE79DF80B00172148434CF21D7104
:10727000C1F67141A0FB01109DF80A100844019964
:107280000844013900EB910048F21F52C5F2EB129D
:10729000A1FB0221A0EB511000EBD110043044F609
:1072A0002511C2F29241A0FB0121421A01EB5202C8
:1072B0009108C900A1EB9201401A00902BE09DF8C3
:1072C0000B00172148434CF21D71C1F67141A0FB20
:1072D00001109DF80A1008440199084400EB910040
:1072E00048F21F52C5F2EB12A1FB0221A0EB511094
:1072F00000EBD110023044F62511C2F29241A0FBFE
:107300000121421A01EB52029108C900A1EB92013E
:10731000401A0090FFE79DF8000004B0704700009D
:1073200080B584B00390029100208DF80700039887
:10733000FFF7D6FE20B1FFE701208DF8070013E02C
:10734000BDF80A00039909680862BDF808000399AE
:10735000096848620398FFF7EFFE20B1FFE70120BC
:107360008DF80700FFE7FFE79DF8070004B080BD38
:1073700080B584B00390029100208DF80700039837
:10738000FFF7AEFE20B1FFE701208DF8070013E004
:10739000BDF80A00039909688861BDF808000399DF
:1073A0000968C8610398FFF7C7FE20B1FFE7012015
:1073B0008DF80700FFE7FFE79DF8070004B080BDE8
:1073C000704700007047000080B596B00CA801908F
:1073D0002821F8F778FF0198002202920B920A9276
:1073E000099208920792069205920492039209214B
:1073F0000C914FF480310D910E9201221092129255
:107400000222139214914FF4E0111591FBF724F925
:1074100018B1FFE7F9F79AFCFFE70F200790022168
:107420000891002009904FF480620A920B9007A8FF
:10743000FAF734FF18B1FFE7F9F788FCFFE70320FC
:1074400003904FF4007004904FF40040059003A89F
:10745000FAF740FE18B1FFE7F9F778FCFFE716B03E
:1074600080BD00007047000080B541F23070C2F26C
:107470000000FCF773FA80BD80B541F23070C2F2B3
:107480000000FCF76BFA80BD80B541F23070C2F2AB
:107490000000FCF763FA80BD80B541F23070C2F2A3
:1074A0000000FCF75BFA80BD80B541F29460C2F247
:1074B0000000FFF7BFFB80BD80B541F2C070C2F293
:1074C0000000FCF74BFA40F20400C2F20000007822
:1074D00038B1FFE740F20401C2F200010020087059
:1074E000FFE780BD83B00290019102980068009090
:1074F000029842F60041C4F20101884215D0FFE72C
:107500000298B0F1804F10D0FFE7029840F200419E
:10751000C4F20001884208D0FFE7029840F600015B
:10752000C4F2000188420AD1FFE7009820F0700001
:10753000009001984168009808430090FFE7029886
:1075400042F60041C4F20101884215D0FFE70298DB
:10755000B0F1804F10D0FFE7029840F20041C4F232
:107560000001884208D0FFE7029840F60001C4F20B
:10757000000188420AD1FFE7009820F44070009093
:107580000198C168009808430090FFE7009820F038
:1075900080000199496908430090009802990860A9
:1075A000019880680299C86201980068029988620F
:1075B000029842F60041C4F20101884205D1FFE77A
:1075C0000198006902990863FFE702990120486168
:1075D00002980069C00730B1FFE70299086920F0FE
:1075E00001000861FFE703B07047000085B0049018
:1075F000039102920193049880680090009820F40F
:107600007F40009003980299019A41EA02210143C8
:1076100000980843009000980499886005B070476E
:1076200083B002900191029880680090009820F049
:107630007000009001980099084340F00700009006
:1076400000980299886003B07047000085B00490EC
:10765000039102920498006A00900499086A20F04D
:1076600001000862049880690190019820F0F00000
:1076700001900299019840EA01100190009820F0D1
:107680000A0000900399009808430090019804991B
:10769000886100980499086205B0704785B004902D
:1076A000039102920498006A00900499086A20F0FD
:1076B00010000862049880690190019820F47040DD
:1076C00001900299019840EA01300190009820F061
:1076D000A00000900399009840EA011000900198E2
:1076E0000499886100980499086205B07047000009
:1076F00080B582B001900198406A00900099002006
:10770000C8850099C8840098FCF710FC02B080BDC1
:1077100084B00390FFE7FFE70398006850E8030F89
:1077200020F490700290FFE702990398026842E803
:1077300003100028F0D1FFE7FFE7FFE7FFE703981A
:10774000006850E8050F20F001000190FFE7019963
:107750000398026842E805100028F0D1FFE7FFE730
:107760000398006B012814D1FFE7FFE7FFE70398B8
:10777000006850E8030F20F010000090FFE7009928
:107780000398026842E803100028F0D1FFE7FFE702
:10779000FFE70399202081F8420003990020086345
:1077A00004B0704780B582B0019001980168C86844
:1077B00020F04000C8600199202081F84100019824
:1077C000FCF7ECFE002002B080BD000080B586B062
:1077D0000490049890F84200222840F0A480FFE72B
:1077E00004988068B0F5805F15D1FFE704980069C0
:1077F00088B9FFE7002003900498806A02900498FB
:10780000006840686FF35F20029908800499886AD5
:107810000230886225E00498806A0390002002907C
:1078200004988068B0F5805F08D0FFE7049880680E
:1078300050B9FFE70498006930B9FFE70498006881
:1078400040680399087007E004980068406800F0F9
:107850007F0003990870FFE70499886A0130886205
:10786000FFE70499C88D0138C8850004002856D167
:10787000FFE704980168C86820F02000C8600498F9
:107880000168C86820F48070C8600498016848697D
:1078900020F0010048610499202081F842000499F9
:1078A000002048630498006B012830D1FFE7049959
:1078B00000200863FFE7FFE70498006850E8030F23
:1078C00020F010000190FFE701990498026842E857
:1078D00003100028F0D1FFE7FFE704980068006874
:1078E000C00600280ED5FFE7FFE7002000900498AF
:1078F0000068006800900498006840680090009854
:10790000FFE7FFE70498818DFCF754F903E0049842
:10791000FCF706FEFFE700208DF8170007E00020C7
:107920008DF8170003E002208DF81700FFE79DF89F
:10793000170006B080BD000080B584B003900398A6
:107940000068006920F44050039A1168D26810431F
:107950000861039988680A694969104308430290DD
:1079600003980068C06841F20C618843029908439B
:1079700003990968C86003980068406920F4407062
:10798000039A11689269104348610398006843F6AE
:107990000001C4F20101884204D1FFE7FAF7ECFDCF
:1079A000019003E0FAF7D6FD0190FFE70198192155
:1079B0004843039A116852689200B0FBF2FC48F207
:1079C0001F52C5F2EB12ACFB02304309642003FBEB
:1079D00010CC322000EB0C10A0FB0202F02000EAD9
:1079E000521000EB0310C2F343121044886004B03D
:1079F00080BD000083B002900191ADF80220019893
:107A000002998862BDF8020002998885BDF80200DB
:107A10000299C8850299002048640299222081F8C1
:107A200042000298006938B1FFE702980168C8680F
:107A300040F48070C860FFE702980168486940F030
:107A40000100486102980168C86840F02000C860E1
:107A5000002003B07047000083B00190019890F8B7
:107A6000410021283AD1FFE701988068B0F5805F96
:107A700013D1FFE70198006978B9FFE70198006A20
:107A80000090009800886FF35F20019909684860B2
:107A90000199086A0230086208E0019A106A411CE4
:107AA00011620078019909684860FFE70199C88C64
:107AB0000138C884000468B9FFE701980168C86804
:107AC00020F08000C86001980168C86840F040005C
:107AD000C860FFE700208DF80B0003E002208DF85E
:107AE0000B00FFE79DF80B0003B0704780B541F233
:107AF0009460C2F20000FFF7A9F980BDFFE7FEE73E
:107B000081B08DF803009DF9030000280ED4FFE733
:107B10009DF9031001F01F02012090404A094EF226
:107B20000011CEF2000141F82200FFE701B07047DA
:107B30004EF60C50CEF200000068C0F302207047F1
:107B400082B08DF8070000919DF9070000280AD443
:107B5000FFE7009800019DF907104EF20042CEF2B7
:107B6000000288540BE0009800019DF8071001F016
:107B70000F014EF61452CEF200028854FFE702B015
:107B80007047000083B00290029800F00700009058
:107B90004EF60C51CEF200010868019001984FF6A4
:107BA000FF02104001900198009A40EA0220002252
:107BB000C0F2FA52104301900198086003B0704778
:107BC00080B582B00190009140F21021C2F2000114
:107BD000FF20087040F21121C2F200010870FFE797
:107BE0000098411E009138B3FFE740F21023C2F223
:107BF0000003187801994A1C01920978414042F229
:107C00008020C2F20000016040F21121C2F20001A6
:107C10000A78D0F800E040F2050CC2F2000C1CF823
:107C20000EC082EA0C021A70026840F20510C2F21D
:107C30000000805C0870D3E740F21020C2F2000020
:107C4000007840F21121C2F20001097840EA0120D7
:107C500002B080BD83B00290019100200090FFE748
:107C600000980199884245DAFFE7009B41F65500EC
:107C7000C2F2000050F83310029AC3EBC30342F87B
:107C80002310009A00EBC20040680299C2EBC202C6
:107C900001EB82014860009A501C0299C2EBC202BB
:107CA00001EB8201088302980099C1EBC10100EB4E
:107CB00081010120888102980099C1EBC10100EB8C
:107CC00081011620887302980099C1EBC10100EB75
:107CD00081011220087502980099C1EBC10100EBE7
:107CE0008101487D40F001004875FFE700980130B0
:107CF0000090B5E703B0704780B584B00390ADF84D
:107D00000A108DF80920ADF8063000200090FFE73A
:107D100000989DF80910884212DAFFE7BDF80A10B2
:107D2000012000FA01F20399C8685040C860BDF80C
:107D30000600F9F78FFCFFE7009801300090E7E7B5
:107D400004B080BD80B590B000200B900F90FAF782
:107D500005F8FFF739FBFEF715F8FEF749F9FEF7CE
:107D6000CDF9FEF789F9FDF7B5FFFDF7E7FFFEF75F
:107D7000A9F8FEF7CBF8FEF713F941F20000C4F2C0
:107D800001000D210A223223FFF7B6FF41F2946071
:107D9000C2F20000099041F60801C2F2000141F26E
:107DA0007872C2F20002FDF721FF0B9B09980321B4
:107DB00041F28832FDF7D8FE0B990998FDF74CFF88
:107DC0000B988DF83B0041F23070C2F20000F8F7DA
:107DD00009FE00F09DFA41F22C60C2F200000A9008
:107DE0000068C17A41F63870C2F20000FFF732FF36
:107DF0000A990B980968C97A40F27832C2F20002F7
:107E0000A2F860190D90FFE70D98FE280BDCFFE744
:107E10000D9841F2D841C2F200010854FFE70D98D5
:107E200001300D90F0E7FFE741F63871C2F2000132
:107E3000059101200790087540F27830C2F20000E9
:107E4000049041F2D441C2F200010391F8F786FF99
:107E50000399049841F22C62C2F2000206920023B8
:107E60000893F8F70BFB00F0B3FA06990598096838
:107E7000C97AFFF7EFFE06980799089AF8F700FF0E
:107E800008980C90FFE70C9841F22C61C2F20001B7
:107E90000968C97A884260DAFFE70C98C0EBC00134
:107EA00041F6A800C2F2000010F831008008C007B7
:107EB00068B1FFE70C98C0EBC00141F6A800C2F220
:107EC000000000EBC101488801304880FFE70C98B2
:107ED000C0EBC00141F6A800C2F20000019000EB27
:107EE000C100F8F70DFE01980C990291C1EBC10198
:107EF00000EBC100006A0021C4F2201100F084FCF4
:107F000000F0D2FB029A014640F27830C2F2000043
:107F100020F8121090F86409C0F3001141F65400E3
:107F2000C2F200000170007848B1FFE740F60C0192
:107F3000C4F20101086840F48060086008E040F67F
:107F40000C01C4F20101086820F480600860FFE7BA
:107F5000FFE70C9801300C9095E765E785B0049039
:107F6000039100200290FFE702980399884280F273
:107F7000CB81FFE700200190FFE7019841F22C61DF
:107F8000C2F200010968C97A884280F2B881FFE72D
:107F9000019800900F2800F2AD810099DFE811F000
:107FA0001000290043005D0077009100AB00C50080
:107FB000DD00F60010012A0144015E017801920102
:107FC0000299019800EB0110C0EBC00241F6A80035
:107FD000C2F2000010F8320000F00102049800EB39
:107FE000410191F8720900F0FE00104481F8720915
:107FF00080E10299019800EB0110C0EBC00241F64C
:10800000A800C2F2000010F8320000F0010204984B
:1080100000EB410191F8720900F0FD0040EA4200D6
:1080200081F8720966E10299019800EB0110C0EB3A
:10803000C00241F6A800C2F2000010F8320000F0C1
:108040000102049800EB410191F8720900F0FB0075
:1080500040EA820081F872094CE10299019800EB34
:108060000110C0EBC00241F6A800C2F2000010F8F7
:10807000320000F00102049800EB410191F872090E
:1080800000F0F70040EAC20081F8720932E102997B
:10809000019800EB0110C0EBC00241F6A800C2F24B
:1080A000000010F8320000F00102049800EB4101DA
:1080B00091F8720900F0EF0040EA021081F87209AD
:1080C00018E10299019800EB0110C0EBC00241F6E3
:1080D000A800C2F2000010F8320000F0010204987B
:1080E00000EB410191F8720900F0DF0040EA421014
:1080F00081F87209FEE00299019800EB0110C0EBD3
:10810000C00241F6A800C2F2000010F8320000F0F0
:108110000102049800EB410191F8720900F0BF00E0
:1081200040EA821081F87209E4E00299019800EBBC
:108130000110C0EBC00241F6A800C2F2000010F826
:108140003220049800EB410191F8720900F07F00A1
:1081500040EAC21081F87209CCE00299019800EB64
:108160000110C0EBC00241F6A800C2F2000010F8F6
:10817000320000F00102049800EB410191F873090C
:1081800000F0FE00104481F87309B3E002990198F1
:1081900000EB0110C0EBC00241F6A800C2F20000E3
:1081A00010F8320000F00102049800EB410191F850
:1081B000730900F0FD0040EA420081F8730999E07C
:1081C0000299019800EB0110C0EBC00241F6A80033
:1081D000C2F2000010F8320000F00102049800EB37
:1081E000410191F8730900F0FB0040EA820081F838
:1081F00073097FE00299019800EB0110C0EBC00207
:1082000041F6A800C2F2000010F8320000F00102AE
:10821000049800EB410191F8730900F0F70040EA7F
:10822000C20081F8730965E00299019800EB011022
:10823000C0EBC00241F6A800C2F2000010F8320004
:1082400000F00102049800EB410191F8730900F07D
:10825000EF0040EA021081F873094BE0029901989F
:1082600000EB0110C0EBC00241F6A800C2F2000012
:1082700010F8320000F00102049800EB410191F87F
:10828000730900F0DF0040EA421081F8730931E021
:108290000299019800EB0110C0EBC00241F6A80062
:1082A000C2F2000010F8320000F00102049800EB66
:1082B000410191F8730900F0BF0040EA821081F893
:1082C000730917E00299019800EB0110C0EBC0029E
:1082D00041F6A800C2F2000010F83220049800EB2A
:1082E000410191F8730900F07F0040EAC21081F863
:1082F0007309FFE7FFE70198013001903DE6FFE7D2
:108300000298013002902FE6002005B0704700006F
:1083100080B582B000200190FFE7019841F22C6106
:10832000C2F200010968C97A88424EDAFFE7019972
:10833000CB17C1EBC10241F6A800C2F2000000EB6E
:10834000C202936251620199C1EBC10100EBC1020B
:1083500040F63541C0F60001C2F82D100199C1EB7D
:10836000C10100EBC1021F2182F82C100199C1EB61
:10837000C10100EBC1020021C4F2A0119160019B78
:1083800040F27831C2F2000101F69412142122F871
:1083900013100199C1EBC10100EBC10301219981C7
:1083A000019B02EB4302A2F8C8100199C1EBC10185
:1083B00000EBC10141F22C60C2F20000F8F7ECFAC8
:1083C000FFE7019801300190A7E702B080BD0000EF
:1083D00080B586B000200590FFE7059841F22C613A
:1083E000C2F200010968C97A884280F28D80FFE7F5
:1083F0000598C0EBC00141F6A800C2F2000000EBF6
:10840000C10081680391016A0491808900F068F9D4
:108410000146039800F0C4FA0146049800F0EFF812
:10842000B0B9FFE70599012000FA01F340F2783175
:10843000C2F20001B1F886291A43A1F88629059AEB
:1084400000FA02F2B1F882099043A1F8820956E0DD
:108450000598C0EBC00141F6A800C2F2000000EB95
:10846000C10081680191016A0291808900F038F9A8
:108470000146019800F04CF80146029800F0C6F859
:10848000B0B9FFE70599012000FA01F340F2783115
:10849000C2F20001B1F886299A43A1F88629059A0B
:1084A00000FA02F2B1F882091043A1F8820925E02E
:1084B0000598C0EBC00141F6A800C2F2000000EB35
:1084C000C1008168006A00F085F8B0B1FFE7059946
:1084D000012000FA01F340F27831C2F20001B1F854
:1084E00082299A43A1F88229059A00FA02F2B1F88A
:1084F00086099043A1F88609FFE7FFE7FFE7FFE75A
:1085000005980130059068E7002006B080BD0000A6
:1085100090EA010F48BF81F0004100F14882421A01
:108520003CBF801A89184FEAD052A2EBD1534FF0CA
:108530007F4C1CEA410F18BF9CEA026F00F03B80A1
:108540004FF0004C4CEA00204CEA012121FA03FCD8
:1085500010EB0C0C1ED202F1FF325FEA1C2040EB44
:10856000C25038BF70471CF07F0F4FEA400C18BF55
:10857000BCF17F4F38BF7047C3F12003994008BF5B
:1085800020F00100BCF17F4F38BF7047A0F1C04020
:1085900000F001BA4FEA3C00000A40EBC25028BF8D
:1085A0001CF0FF0F4FEA400CE6D018BFBCF17F4F24
:1085B00038BF7047EAE79CEA026F05D010EA5C0F0B
:1085C00008BF00F00040704710B500F09EF900BFF2
:1085D00064FBBE3E10B500F033F80CBF0120002054
:1085E00010BD10B500F02CF814BF0120002010BD04
:1085F00010B500F0A1F88CBF0120002010BD10B50F
:1086000000F09AF82CBF0120002010BD10B500F03A
:10861000C7F894BF0120002010BD10B500F0C0F8CD
:1086200034BF0120002010BD401058BFC0F14040B1
:10863000491058BFC1F140418142EFF300807047BB
:1086400050EA010C00F113801CF5000F58BFBCF577
:10865000000F01D48842704707D710F5000F58BFAC
:1086600011F5000F15D488427047894270471CF5F8
:10867000000F04D5BCF5000FF7D5814270474FF0CD
:10868000807C1CEB400F38BF1CEB410F01D28142B4
:10869000704710B500F039F9922449004FF00050AE
:1086A0004FF08051FFF7C0BF41000B0ED3F19E0287
:1086B00008D950F400034FEA032323FA02F048BF1D
:1086C0004042704710B500F020F900BF4992248065
:1086D000002070476FF0004282EA200070470000DF
:1086E00010F0004148BF4042B0FA80F310FA03F2A4
:1086F000C3F19D030BD051EAC35101EB1220530685
:1087000038BF704700F1010008BF20F0010070473A
:10871000B0FA80F310FA03F2C3F19D030AD0D90531
:1087200001EB1220530638BF704700F1010008BF6B
:1087300020F001007047000050EA010C00F11380A6
:108740001CF5000F58BFBCF5000F01D488427047DC
:1087500007D710F5000F58BF11F5000F15D4884248
:108760007047894270471CF5000F04D5BCF5000F17
:10877000F7D5814270474FF0807C1CEB400F38BF2B
:108780001CEB410F01D28142704710B500F0BDF8DB
:10879000922449004FF080504FF00051FFF744BF42
:1087A00050EA010C00F113801CF5000F58BFBCF516
:1087B000000F01D48842704707D710F5000F58BF4B
:1087C00011F5000F15D488427047894270471CF597
:1087D000000F04D5BCF5000FF7D5814270474FF06C
:1087E000807C1CEB400F38BF1CEB410F01D2814253
:1087F000704710B500F089F8922449004FF00050FE
:108800004FF08051FFF710BF4FF47F0C1CEAD012DD
:108810001EBF1CEAD11392EA0C0F93EA0C0F00F072
:10882000478090EA010F48BF42F480724FF0004C3D
:108830004CEA00204CEA012102EB0302A0FB0113E9
:10884000A2F50002002918BF43F001035B0028BF16
:108850004FEA330342EB22425FEA132C4CEBC25047
:108860002EBFBCEB436FB2F57C0F70474FEA036C31
:10887000BCF1004F08BF20F00100B2F57C0F38BFFB
:1088800070470BD582F0FF0212F5803FC8BF7047DA
:1088900000F1C040D8BF00F00040704700F5000C68
:1088A0005FEA4C0C48BF7047B0F1C04000F073B8AD
:1088B0000CEAD11390EA010F48BF42F4807262457E
:1088C00038BF634504D280EA010000F000407047E1
:1088D00010B500F01AF800BF8900013E00F007B89B
:1088E00000F009B85FEA410C5FEA1C6C08D080EA2E
:1088F000010000F050B85FEA400C5FEA1C6CF6D152
:108900004FF00040A0F5800070470EF1020E2EF0EF
:10891000030E5EF8044B244204D44FEA4102B2F144
:108920007F4F11D84FEA4003B3F17F4F0CD80ED1DF
:108930004FEAD07C0CEB4C0C0CF1020CB2F17F4FE7
:1089400008BF4CEBD17C04E04FF0080C01E04FEA8B
:10895000D17C0CEB4C0324FA03F404F00704B4F1CB
:10896000040C06D20EEB840CBDE810404CF0010C58
:108970006047DFE80CF0070802024FF00040A0F566
:10898000800010BD0846420018BFD2F1807288BF37
:1089900000F0004010BDFF2141EAD050C0057047F3
:1089A00090EA010F48BF81F000413FF5B8AD421A8F
:1089B00004D882F00042A0EB020011444FEAD052EA
:1089C000A2EBD1534FF07F4C1CEA410F18BF9CEA39
:1089D000026F4AD04FF0004C4CEA00204CEA0121D3
:1089E00021FA03FCB0EB0C0C0FD412F0FE0F36D0C2
:1089F0005FEA4C001DD5001240EBC25038BF7047F3
:108A00001CF03F0F18BF70470BE05FEA1C20A2F17B
:108A1000010240EBC25038BF70471CF07F0F18BFF7
:108A20007047C3F12003994014BF401E20F001009D
:108A300070474FEA1223800808BF7047B0FA80FCE5
:108A4000A2EB0C02CCF1280C60FA0CF093EA122F86
:108A500004BF00EBC25070474FEAC3707047130A5F
:108A60005FEADC1008BF7047F6E79CEA026F04D0AB
:108A700010EA5C0F08BF0020704710B5FFF745FFF4
:108A800040DFF63E81F0004070470000000000002B
:108A900000000102030406070809000000000102AB
:108AA000030402030405060708090A0B0C0D0E0F48
:108AB0001010010202030405060708090A0B0C0D39
:108AC0000E0F101001024E494F2D313200000000F0
:108AD000F08A000800000020180200005001000881
:108AE000308C00081802002070260000B801000831
:108AF000200E00127A000100C1814001C0804104B3
:108B0000610C2108E118A11C011A30011638013648
:108B100060012E70012F6000FF00C0C101C303027D
:108B2000C2C60607C705C5C404CC0C0DCD0FCFCEF9
:108B30000E0ACACB0BC90908C8D81819D91BDBDA29
:108B40001A1EDEDF1FDD1D1CDC14D4D515D7171649
:108B5000D6D21213D311D1D010F03031F133F3F259
:108B60003236F6F737F53534F43CFCFD3DFF3F3E39
:108B7000FEFA3A3BFB39F9F83828E8E929EB2B2AC9
:108B8000EAEE2E2FEF2DEDEC2CE42425E527E7E689
:108B90002622E2E323E12120E0A06061A163A3A2F9
:108BA0006266A6A767A56564A46CACAD6DAF6F6E79
:108BB000AEAA6A6BAB69A9A86878B8B979BB7B7AA9
:108BC000BABE7E7FBF7DBDBC7CB47475B577B7B6C9
:108BD0007672B2B373B17170B05090915193535299
:108BE0009296565797559594549C5C5D9D5F9F9EB9
:108BF0005E5A9A9B5B99595898884849894B8B8A49
:108C00004A4E8E8F4F8D4D4C8C4484854587474608
:108C100086824243834181801006400000001C048C
:108C2000124804000900FFFF0100100000000000CE
:04000005080000ED02
:00000001FF
